:10000000A2C20000D1C20000CFC20000CDC20000D9
:10001000CBC20000C9C20000C7C20000C5C20000B8
:10002000C3C20000C1C20000BFC20000BDC20000C8
:10003000BBC20000B9C20000B7C20000B5C20000D8
:10004000B3C200000C94DF14AFC20000ADC20000C8
:100050000C940C15A9C20000A7C200000C94CF3B61
:10006000A3C200000C9417130C94EE129DC2000062
:100070009BC2000099C2000097C2000095C2000018
:100080000C94B21491C200008FC200008DC2000017
:100090008BC2000089C2000087C2000085C2000038
:1000A00083C2000081C200000C9485147DC2000050
:1000B0007BC2000079C2000077C200000C94581483
:1000C00073C2000071C200006FC200006DC2000068
:1000D0006BC2000069C2000067C2000065C2000078
:1000E00063C20000ED17FA1703180C18191822182C
:1000F000BE1BBE1BBE1BBE1BBE1B2F183C184918C7
:10010000BE1B56185F18681875187E188718901847
:100110009918A218BE1BAB18B418BD18BE1BBE1B85
:10012000BE1BC618CF18D818BE1BBE1BE118EE1890
:10013000BE1BBE1BBE1BFB1808191519BE1B2219BE
:100140002B193419BE1BBE1BBE1B3D1946194F1976
:10015000BE1B5C1969197619BE1BBE1BBE1B831919
:1001600090199D19BE1BAA19B719C419BE1BBE1B35
:10017000BE1BD119DE19EB19BE1BF819011A0A1A98
:10018000BE1BBE1BBE1BBE1BBE1BBE1BBE1BBE1BA7
:10019000BE1BBE1BBE1BBE1BBE1BBE1BBE1BBE1B97
:1001A000BE1BBE1BBE1BBE1BBE1BBE1BBE1B2E1A18
:1001B000371A401ABE1B491A521A5B1ABE1BBE1BC5
:1001C000BE1B641A711A7E1ABE1B8B1A981AA51AC6
:1001D000BE1BBE1BBE1BB21ABF1ACC1ABE1BD91A3D
:1001E000E21AEB1ABE1BBE1BBE1BF41AFD1A061B3D
:1001F000BE1BBE1BBE1BBE1BBE1BBE1BBE1BBE1B37
:10020000BE1BBE1BBE1B131A1C1A251ABE1BBE1B0F
:10021000BE1BBE1BBE1BBE1BBE1BBE1BBE1BBE1B16
:10022000BE1BBE1BBE1BBE1BBE1BBE1BBE1BBE1B06
:10023000BE1BBE1BBE1BBE1BBE1BBE1BBE1BBE1BF6
:10024000BE1BBE1BBE1BBE1BBE1BBE1BBE1BBE1BE6
:10025000BE1BBE1BBE1BBE1BBE1BBE1BBE1BBE1BD6
:10026000BE1BBE1BBE1BBE1BBE1BBE1BBE1BBE1BC6
:10027000BE1BBE1BBE1B0F1B181B251BBE1B321B30
:100280003B1B481BBE1BBE1BBE1B551B5E1B6B1BBB
:10029000BE1B781B811B8E1BBE1BBE1BBE1B9B1B6C
:1002A000A41BB11BE325E825ED25F72501267A26B9
:1002B0000B2613261B2625262F26392648265226AE
:1002C0007A265C2666267026E738EA38D938DD3883
:1002D000E3382139EE38F238F838FC38003906397D
:1002E0000A390E392139143918391C394E414E4911
:1002F0004E495459494E46CDCCCC3D0AD7233C17E4
:10030000B7D13877CC2B329595E6241FB14F0A0030
:100310000020410000C84200401C4620BCBE4CCA20
:100320001B0E5AAEC59D7400407A10F35A00A0729D
:100330004E18090010A5D4E80000E8764817000020
:10034000E40B54020000CA9A3B000000E1F50500EE
:100350000080969800000040420F000000A0860137
:10036000000000102700000000E803000000006407
:1003700000000000000A0000000000010000000072
:10038000002C76D888DC674F0823DFC1DFAE59E147
:10039000B1B796E5E3E453C63AE651997696E8E6B6
:1003A000C28426EB898C9B62ED407C6FFCEFBC9C89
:1003B0009F40F2BAA56FA5F490055A2AF75C936B9B
:1003C0006CF9676DC11BFCE0E40D47FEF520E6B556
:1003D00000D0ED902E0300943577050080841E0830
:1003E0000000204E0A000000C80C333333330F984E
:1003F0006E12831141EF8D2114893BE65516CFFE15
:10040000E6DB18D1844B381BF77C1D901DA4BBE4A0
:1004100024203284725E228100C9F124ECA1E53DE2
:100420002700002100240027002A002D003000337F
:100430000001010000040107010A0100002200255B
:100440000028002B002E00310034000201000005BE
:100450000108010B01000020002300260029002CC8
:10046000002F003200000100000301060109010510
:10047000050505070508080808020202020A0A081D
:100480000804040404010101010101010103030343
:100490000303030303040707070C0C0C0C0C0C0CE0
:1004A0000C0202020206060606060606060B0B0BE7
:1004B0000B0B0B0B0B010210202008081020401022
:1004C0002040800201020108040201010204081018
:1004D0002040808040201008040201800402018036
:1004E000402010080402010804020101020408105F
:1004F000204080010204081020408000000A0B0206
:10050000090C0D0E080703040100000000000000A4
:1005100000000000000000000000000000000000DB
:100520000000000000000012111000000000000098
:1005300000000000000000000000000000000000BB
:10054000000041463C4611241FBECFEFD1E2DEBF82
:10055000CDBF00E00CBF17E0A0E0B2E0ECEFFFE998
:1005600000E00BBF02C007900D92A234B107D9F78B
:100570002DE0A2E4B7E001C01D92AA34B207E1F772
:1005800012E0C2EAD2E000E006C021970109802F04
:10059000FE010E94E54EC13AD10780E00807A9F7A5
:1005A0000E94193C0C94ED4F2BCD0C946B470C948E
:1005B0006B470C946B470C946B470C946B470C94F3
:1005C0006B470C946B470C946B470C946B470C94E3
:1005D0006B470C946B470C946B470C946B470C94D3
:1005E0006B470C946B470C946B470C946B470F93C1
:1005F0001F93CF93DF93FB0102A913A9C68DD78D5B
:100600000E948726A801BE010E94342580E090E068
:10061000DF91CF911F910F910895662319F08DEA14
:1006200093E002C086EA93E00C9459390F931F932C
:10063000CF93DF93FB0102A113A1C68DD78D0E943A
:10064000C524C530D105E1F064F4249771F564E068
:1006500070E08DE29DE00E94D013B8018DE29DE034
:1006600022C0C630D105B1F02B97F9F46BE070E0F1
:1006700086E39DE00E94D013B80186E39DE013C09D
:1006800065E070E080E39DE00E94D013B80180E354
:100690009DE009C066E070E083E39DE00E94D01316
:1006A000B80183E39DE00E944D1380E090E0DF916C
:1006B000CF911F910F910895EF92FF920F931F9387
:1006C000CF93DF93FB01E2A8F3A802A113A1C68D8B
:1006D000D78D0E9487269701A801BE010E94A02500
:1006E00080E090E0DF91CF911F910F91FF90EF900C
:1006F00008954F925F926F927F92AF92BF92CF9286
:10070000DF92EF92FF920F931F93CF93DF93FB0142
:10071000E2A8F3A846A457A460A871A8C6A0D7A0D1
:10072000A2A0B3A0068D178D0E948726EC01970129
:10073000A501B8010E94A025C301B2010E948B3B14
:100740009701A601B801CE010E94A02580E090E0AB
:10075000DF91CF911F910F91FF90EF90DF90CF909D
:10076000BF90AF907F906F905F904F900895CF9320
:10077000DF93FB01D2A9C68D0E9487266D2F8C2F97
:100780000E94443B80E090E0DF91CF910895CF93A9
:10079000DF93FB01C68DD78D0E94691EBE010E94AA
:1007A000271E80E090E0DF91CF910895CF92DF92F5
:1007B000EF92FF920F931F93CF93DF93FB01C2A0A1
:1007C000D3A0E4A0F5A0068D178D0E94691EEC0150
:1007D0008A819B818F30F7E29F0724F401969B83E7
:1007E0008A8302C01B821A82B801CE010E94391D81
:1007F0008823B1F0F801EE0FFF1FEE0FFF1FEA5A3A
:10080000F84FC082D182E282F382A7019601B8013B
:10081000CE010E94EA1DB801CE010E94271E04C02D
:100820008DE994E00E9459390E9408250E94D8243D
:1008300080E090E0DF91CF911F910F91FF90EF90BA
:10084000DF90CF9008958F929F92AF92BF92CF92F8
:10085000DF92EF92FF920F931F930E94AC2462E00D
:1008600070E00E94AC33892BC9F40E94AC2421E0D3
:100870002F931F921F921F921F92812C912CA12CBB
:10088000B12CC12CD12C760197018601B701A601AC
:1008900037D30F900F900F900F900F9080E090E063
:1008A0001F910F91FF90EF90DF90CF90BF90AF908E
:1008B0009F908F9008958F929F92AF92BF92CF9208
:1008C000DF92EF92FF920F931F930E94AC2461E09E
:1008D00070E00E94AC33892BC9F40E94AC241F92B3
:1008E00021E02F931F921F921F92812C912CA12CFB
:1008F000B12CC12CD12C760197018601B701A6013C
:10090000FFD20F900F900F900F900F9080E090E02B
:100910001F910F91FF90EF90DF90CF90BF90AF901D
:100920009F908F9008958F929F92AF92BF92CF9297
:10093000DF92EF92FF920F931F930E94AC2460E02E
:1009400070E00E94AC33892BC9F40E94AC241F9242
:100950001F9221E02F931F921F92812C912CA12C8A
:10096000B12CC12CD12C760197018601B701A601CB
:10097000C7D20F900F900F900F900F9080E090E0F3
:100980001F910F91FF90EF90DF90CF90BF90AF90AD
:100990009F908F9008958F929F92AF92BF92CF9227
:1009A000DF92EF92FF920F931F930E94AC2421E0FD
:1009B0002F931F921F921F921F92812C912CA12C7A
:1009C000B12CC12CD12C760197018601B701A6016B
:1009D00097D20F900F900F900F900F9080E090E0C3
:1009E0001F910F91FF90EF90DF90CF90BF90AF904D
:1009F0009F908F9008958F929F92AF92BF92CF92C7
:100A0000DF92EF92FF920F931F930E94AC241F92EC
:100A100021E02F931F921F921F92812C912CA12CC9
:100A2000B12CC12CD12C760197018601B701A6010A
:100A300067D20F900F900F900F900F9080E090E092
:100A40001F910F91FF90EF90DF90CF90BF90AF90EC
:100A50009F908F9008958F929F92AF92BF92CF9266
:100A6000DF92EF92FF920F931F930E94AC241F928C
:100A70001F9221E02F931F921F92812C912CA12C69
:100A8000B12CC12CD12C760197018601B701A601AA
:100A900037D20F900F900F900F900F9080E090E062
:100AA0001F910F91FF90EF90DF90CF90BF90AF908C
:100AB0009F908F900895089508950895089508953A
:100AC000089508950895089508950895089508953E
:100AD0000895089508950895EF92FF920F931F933C
:100AE000CF93DF93CDB7DEB72E970FB6F894DEBF66
:100AF0000FBECDBF8C010E948B396FEB74E0C80133
:100B00000E94DA126091460770914707809148076A
:100B1000909149072AE0AE014F5F5F4F7A010E9432
:100B20002B48F70101900020E9F73197AF014E19EA
:100B30005F09B701C8010E94AD126CE973E0C801FA
:100B40000E94DA12C8012E960FB6F894DEBF0FBECF
:100B5000CDBFDF91CF911F910F91FF90EF9008953E
:100B60008FEB94E00E9459396091460770914707D6
:100B700080914807909149070E94F9398CE993E0E8
:100B80000C9459390F931F93CF93DF93EC0182ECB0
:100B900094E00E94593986EC94E00E94593902EEA3
:100BA0001BE0F8016081CE0138DD8AEC94E00E9400
:100BB0005939F8016181CE0130DD8EEC94E00E945C
:100BC0005939F8016281CE0128DD82ED94E00E945E
:100BD0005939F8016381CE0120DD86ED94E00E9451
:100BE0005939F8016481CE0118DD8AED94E00E9444
:100BF0005939F8016581CE0110DDCE01DF91CF9129
:100C00001F910F91ADCFCF92DF92EF92FF92CF93D2
:100C1000DF93EC0188819981AA81BB81181619069E
:100C20001A061B0644F081E090E0A0E0B0E0888363
:100C30009983AA83BB838C819D81AE81BF81181665
:100C400019061A061B0644F081E090E0A0E0B0E02F
:100C50008C839D83AE83BF8388859985AA85BB8558
:100C6000181619061A061B0644F081E090E0A0E071
:100C7000B0E088879987AA87BB878EED94E00E94B1
:100C8000593980EF95E00E94593960914A07709177
:100C90004B0780914C0790914D070E944A4C6B0185
:100CA0007C01688179818A819B810E944A4C9B01E9
:100CB000AC01C701B6010E94384E42E00E94203AC2
:100CC00080E096E00E94593960914E0770914F077D
:100CD00080915007909151070E944A4C6B017C0112
:100CE0006C817D818E819F810E944A4C9B01AC0169
:100CF000C701B6010E94384E42E00E94203A80E1CE
:100D000096E00E9459396091520770915307809183
:100D10005407909155070E944A4C6B017C016885ED
:100D200079858A859B850E944A4C9B01AC01C7014D
:100D3000B6010E94384E42E00E94203ACE01DF9177
:100D4000CF91FF90EF90DF90CF900ACF8091E00B92
:100D50009091E10B892B71F58DE090E00E94D346D4
:100D6000FC01148610924A0710924B0710924C0710
:100D700010924D0710924E0710924F071092500795
:100D80001092510710925207109253071092540775
:100D90001092550710924607109247071092480785
:100DA0001092490710924507109244079093E10B67
:100DB0008093E00B8091E00B9091E10B0895C6DFEA
:100DC00022DF80E090E008950F931F93CF93DF938D
:100DD0000E94691E8C01C0E0D0E0BE01C8010E94E3
:100DE000391D882321F0BE01C8010E94271E2196CB
:100DF000C13ED10591F782EE94E00E945939A6DFF9
:100E0000AFDE80E090E0DF91CF911F910F910895C8
:100E10009DDFFC01148680E090E00895CF93DF937E
:100E200083E00E94EE3AEC0191DF81E0CD2B09F4E2
:100E300080E08093E20B82E00E94EE3AEC0186DFD4
:100E400081E0CD2B09F480E08093E30B8EE00E94DB
:100E5000EE3AEC017BDF81E0CD2B09F480E080935A
:100E6000E40B8FE00E94EE3AEC0170DF81E0CD2BC5
:100E700009F480E08093E50B82E10E94EE3AEC01F8
:100E800065DF81E0CD2B09F480E08093E60B83E100
:100E90000E94EE3AEC015ADF81E0CD2B09F480E0AC
:100EA0008093E70BDF91CF91089586EE94E00E9446
:100EB00059394CDFB3DF4ADF65DE0E94872640E008
:100EC00050E068E070E00E9434250E94872640E0F0
:100ED00050E069E070E00E9434250E94872640E0DF
:100EE00050E06AE070E00E9434250E94872640E0CE
:100EF00050E06DE070E00E94342580E090E00895BD
:100F00002F923F924F925F926F927F928F929F9219
:100F1000AF92BF92CF92DF92EF92FF920F931F9307
:100F2000CF93DF93CDB7DEB7EA970FB6F894DEBF65
:100F30000FBECDBF1C012A013B010B871C872D87EB
:100F40003E8762960EAD1FAD6297FC01E359FD4FDF
:100F500060817181828193810E944A4CA301920138
:100F60000E94A94C0E94A04E6F8F78A389A39AA3D8
:100F7000F101EF58FD4F60817181828193810E9460
:100F80004A4C2B853C854D855E850E94A94C0E946C
:100F9000A04E6FA378A789A79AA7F101EB58FD4F40
:100FA00060817181828193810E944A4CA7019601E0
:100FB0000E94A94C0E94A04E6BA77CA78DA79EA75C
:100FC0000E94C33B6F8B788F898F9A8FF101E2511A
:100FD000FE4F118210823296118210823E96A11429
:100FE000B10461F0C501A0E0B0E0408151816281AF
:100FF000738184179507A607B70714F0A080B18006
:10100000F101EE5FFD4F8114910461F0C401A0E095
:10101000B0E0408151816281738184179507A607F2
:10102000B70714F080809180F101EA5FFD4F011550
:10103000110561F0C801A0E0B0E0408151816281FA
:10104000738184179507A607B70714F000811181F3
:101050009101205F3F4F3C872B87C501A0E0B0E0A6
:10106000F10180A791A7A2A7B3A73101FAE86F0EFB
:10107000711CA12CB12CD30158968D929D92AD92EA
:10108000BC925B972101BCEF4B1ABEEF5B0A20E0DC
:1010900030E0F201008F118F228F338F57DE56DE42
:1010A00055DE54DE20914A0730914B0740914C07A2
:1010B00050914D072F87388B498B5A8B47DE809094
:1010C0004E0790904F07A0905007B09051073EDE1A
:1010D0008091520790915307A0915407B091550702
:1010E0008B8B9C8BAD8BBE8BF101E758FD4F108233
:1010F000118212821382349610821182128213821C
:1011000034961082118212821382349611821082D8
:1011100032961182108232961182108232962F8579
:10112000388949895A89208331834283538334968D
:1011300080829182A282B382349680839183A2833B
:10114000B3836396EFAC63970F8D18A129A13AA1E1
:101150004F85588969897A898B859C850E947B1681
:101160008823E9F085E393E00E94593980EF95E008
:101170000E945939F101EE5AFF4F608171818281DD
:101180009381E55EFD4F20813181428153810E9430
:10119000764DCA01B9010E94F939D8DDE1DC6496C7
:1011A000EFAC64970FA118A529A53AA5B501A40134
:1011B000C3010E947B168823E9F081E393E00E943B
:1011C000593980E096E00E945939F101E453FF4F0C
:1011D0006081718182819381EB55FE4F2081318145
:1011E000428153810E94764DCA01B9010E94F939AA
:1011F000ADDDB6DC6596EFAC65970BA51CA52DA5FE
:101200003EA54B895C896D897E89C2010E947B164F
:101210008823E9F08DE293E00E94593980E196E05D
:101220000E945939F101EA5BFE4F60817181828130
:101230009381E15DFE4F20813181428153810E9483
:10124000764DCA01B9010E94F93980DD89DCD101EE
:1012500051961C92F101E557FF4F1082E658FF4F5F
:101260001082C1010E948931C1010E948D318B859C
:101270009C850E944330C3010E944330C2010E94FA
:101280004330F101EB50FE4FF8A7EFA381E090E06F
:10129000918380837101F9E0EF1AFEEFFF0AD70115
:1012A0008D939C93810107501E4FF8019183808399
:1012B00041E050E06B857C85C1010E946223D7012B
:1012C0004D915C91B301C1010E946223F8014081FC
:1012D0005181B201C1010E94622311E0F101E65285
:1012E000FD4F10838B859C850E946616C3010E946A
:1012F0006616C2010E94661664E670E080E090E027
:101300000E948B3BC1018E509E4FDC011C931196B5
:101310001C93A1014C505E4FFA0110836396FFAD00
:101320006397F1110FC064962FAD6497211105C02A
:1013300065963FAD6597332339F1910121593F4FB0
:10134000F90110826496FFAD6497F11105C0910117
:1013500027513F4FF90110826596FFAD6597F11156
:1013600005C091012D593E4FF901108263962FADB2
:101370006397FC01208364963FAD64973C93659628
:10138000EFAD6597DA01EC938B859C850E949C2DCF
:10139000C3010E949C2DC2010E949C2D8B859C85BF
:1013A0000E947A17C3010E947A17C2010E947A171D
:1013B000CDDCDC011C968C918B8BA12CB12C4101D6
:1013C000BEE08B1ABEEF9B0AF101ED50FE4FF88B89
:1013D000EF8791012C503E4F38A32F8FA1014B5026
:1013E0005E4F5CAB4BABC10189509E4F9EAB8DAB4A
:1013F000D101A750BE4FB8AFAFABE158F140FAAB47
:10140000E9AB2F533F4F3AAF29AF4D5251405CA744
:101410004BA7855B910998AB8FA7D4018C91811163
:101420000AC0EF85F8898081811105C0AF8DB8A110
:101430008C91882319F0BB89BB2321F081010851CD
:101440001E4F4CC34BA95CA96B857C85C1010E94D2
:10145000BB234DA95EA9B301C1010E94BB234FA9C3
:1014600058ADB201C1010E94BB238B859C850E94AF
:10147000462DC3010E94462DC2010E94462DE9A9B6
:10148000FAA98081882331F18B859C850E949C2D4F
:10149000A9ADBAAD8C918823D1F06101B7E5CB1A23
:1014A000BDEFDB0A7101E6E3EE1AEDEFFE0A810102
:1014B00009561D4F910125573D4FA10147585D4FDA
:1014C000B10162587E4F8B859C850E94CB30A9A9C3
:1014D000BAA91C92F101E451FF4F8081882331F1B8
:1014E000C3010E949C2DF101EA54FD4F80818823A5
:1014F000C9F06101B3E5CB1ABDEFDB0A7101E4E38A
:10150000EE1AEDEFFE0A810105561D4F910121579C
:101510003D4FA10143585D4FB10160567E4FC3015D
:101520000E94CB30F101E451FF4F1082F101EA59E2
:10153000FE4F8081882331F1C2010E949C2DF10170
:10154000E954FD4F80818823C9F06101FFE4CF1A7F
:10155000FDEFDF0A710122E3E21A2DEFF20A8101A9
:1015600001561D4F91012D563D4FA1014F575D4F23
:10157000B1016E537E4FC2010E94CB30F101EA5996
:10158000FE4F1082810101591F4FD8018C91882391
:1015900009F43CC0F101ED55FD4F60817181072ECA
:1015A000000C880B990B0E944A4C9B01AC01F10185
:1015B000E758FD4F60817181828193810E94D14EF5
:1015C000181624F5D8011C9264E274E081010C51D4
:1015D0001E4FC801EFD767E275E0C801EBD76CE991
:1015E00073E0C801E7D76396BFAD6397BB2309F4E7
:1015F0006FC3F101E258FE4F108A118A128A138AD2
:10160000E053F1401082118212821382810107514E
:101610001F4FF8018081882309F43CC0E454FE4F39
:1016200060817181072E000C880B990B0E944A4C37
:101630009B01AC01F101E358FD4F60817181828112
:1016400093810E94D14E18162CF5F801108264E2A5
:1016500074E081010C511E4FC801ACD76FE475E0F6
:10166000C801A8D76CE973E0C801A4D76496FFADA0
:101670006497FF2309F430C3F101E056FE4F108A4E
:10168000118A128A138AABA5BCA51D921D921D92C8
:101690001C92139781010D591E4FF80180818823F8
:1016A00009F43CC0EC5BFE4F60817181072E000C99
:1016B000880B990B0E944A4C9B01AC01F101EF573A
:1016C000FD4F60817181828193810E94D14E1816F5
:1016D0002CF5D8011C9264E274E081010C511E4F7C
:1016E000C80168D767E775E0C80164D76CE973E0A3
:1016F000C80160D76596BFAD6597BB2309F4F0C2FA
:10170000F101EE53FE4F108A118A128A138AAFA597
:10171000B8A91D921D921D921C92139760E08B85B3
:101720009C850E94F316882369F0F101E25BFF4F6C
:101730001082118212821382E05DFE4F108A118A9C
:10174000128A138A60E0C3010E94F316882369F0AD
:10175000EBA5FCA51082118212821382F101E056E2
:10176000FE4F108A118A128A138A60E0C2010E9419
:10177000F316882371F0AFA5B8A91D921D921D9292
:101780001C921397F101EE53FE4F108A118A128AB0
:10179000138AF101E159FF4F8081F4018083F10147
:1017A000E751FF4F8081AF85B8898C93E658FF4F92
:1017B0008081EF8DF8A18083F101E25BFF4F2081F2
:1017C0003181428153812BA33CA34DA35EA3ABA5E2
:1017D000BCA58D919D910D90BC91A02D8F83988774
:1017E000A987BA87EFA5F8A9C080D180E280F380ED
:1017F000ADDA2BA13CA14DA15EA120934A07309305
:101800004B0740934C0750934D07A0DA8F81988582
:10181000A985BA8580934E0790934F07A0935007F0
:10182000B093510793DAC0925207D0925307E092D7
:101830005407F0925507C1010E948931D4018C915F
:10184000882309F44AC00E94C33B2F89388D498DF3
:101850005A8D621773078407950760F40E94C33B93
:101860002F89388D498D5A8D621773078407950724
:10187000A0F51EC00E94C33B6B017C012F89388DEF
:10188000498D5A8DC21AD30AE40AF50AF101EF59BB
:10189000FD4F2081318142815381A8EEB3E00E9447
:1018A000924D6C157D058E059F0508F41DC2D6CF9F
:1018B0000E94C33B6B017C01F101EF59FD4F208178
:1018C000318142815381A8EEB3E00E94924D6C15A4
:1018D0007D058E059F0508F407C2AF85B8898C91F8
:1018E000882309F44AC00E94C33B2F89388D498D53
:1018F0005A8D621773078407950760F40E94C33BF3
:101900002F89388D498D5A8D621773078407950783
:10191000A0F51EC00E94C33B6B017C012F89388D4E
:10192000498D5A8DC21AD30AE40AF50AF101EB591E
:10193000FD4F2081318142815381A8EEB3E00E94A6
:10194000924D6C157D058E059F0508F4E0C1D6CF3C
:101950000E94C33B6B017C01F101EB59FD4F2081DB
:10196000318142815381A8EEB3E00E94924D6C1503
:101970007D058E059F0508F4CAC1AF8DB8A18C9175
:10198000882309F44AC00E94C33B2F89388D498DB2
:101990005A8D621773078407950760F40E94C33B52
:1019A0002F89388D498D5A8D6217730784079507E3
:1019B000A0F51EC00E94C33B6B017C012F89388DAE
:1019C000498D5A8DC21AD30AE40AF50AF101E75982
:1019D000FD4F2081318142815381A8EEB3E00E9406
:1019E000924D6C157D058E059F0508F4A3C1D6CFD9
:1019F0000E94C33B6B017C01F101E759FD4F20813F
:101A0000318142815381A8EEB3E00E94924D6C1562
:101A10007D058E059F0508F48DC187EF9BE021D3DE
:101A2000181619065CF587EF9BE0F9D28F7D853497
:101A3000910521F56DEE74E0C1018C519E4FBAD530
:101A400082E693E00E94593981D98AD8F101E1599F
:101A5000FF4F1082E658FF4F1082E658FF4F10826A
:101A6000D4011C92EF85F8891082AF8DB8A11C9229
:101A7000B1E0BB8BAA24A394B12C03C0A114B10480
:101A800071F062E075E0C1018C519E4F93D5F40175
:101A90001082AF85B8891C92EF8DF8A11082C10128
:101AA0000E947438F101E051FE4F808191810196CE
:101AB000918380838D3291400CF4AFCCD101A85139
:101AC000BE4F8D919C911197892B09F0A6CC14964D
:101AD0008D919C91892B09F440C19FCCF8018081A4
:101AE0009181892B21F0C1010E947438F7CF8EE0DB
:101AF00095E00E9459396396FFAD6397FF23F1F09B
:101B0000A114B10439F52B8921113CC08DE193E07A
:101B10000E9459391BD924D864963FAD649733236A
:101B200009F40FC289E193E00E9459390FD918D8FE
:101B300065964FAD6597442351F11CC064965FAD27
:101B40006497552361F0A114B10409F58B898111C3
:101B50001EC0E8CF6496EFAD6497E11118C065969A
:101B60009FAD6597992399F0A114B10481F4AB89D5
:101B7000A1110DC085E193E00E945939E7D80E9478
:101B8000B00505C06496FFAD6497FF2341F385E07F
:101B900090E0EFA1F8A591838083810109501E4F49
:101BA000D8018D939C934101B7E08B1ABEEF9B0A3D
:101BB000F4019183808345E050E06B857C85C10111
:101BC0000E946223D8014D915C91B301C1010E9432
:101BD0006223F40140815181B201C1010E9462235C
:101BE000C1010E949131F101E25BFF4F20813181FF
:101BF000428153812B8F3C8F4D8F5E8FE658FF4F74
:101C000080819181A281B3818F8B988FA98FBA8FA8
:101C1000E658FF4FC080D180E280F38097D82B8DAB
:101C20003C8D4D8D5E8D20934A0730934B0740933A
:101C30004C0750934D078AD88F89988DA98DBA8DFE
:101C400080934E0790934F07A0935007B09351078E
:101C50007DD8C0925207D0925307E0925407F09279
:101C60005507C1010E948931C1010E948D316ED892
:101C70000E940306C1010E94F323AFA1B8A51D92E3
:101C80001C92F80111821082D4011D921C9240E036
:101C900050E06B857C85C1010E946223F801408180
:101CA0005181B301C1010E946223D4014D915C9125
:101CB000B201C1010E946223C1010E949131BB891E
:101CC000BB2309F444C142D821E0FC0124873FC171
:101CD000AA24A394B12C9ACCAA24A394B12CDACC34
:101CE000AA24A394B12C1ACD69E273E081010C51AE
:101CF0001E4FC8015FD46CE973E0C8015BD46FE983
:101D000075E0C80157D422E0A22EB12CE6CD65E2E1
:101D100073E081010C511E4FC8014CD46CE973E093
:101D2000C80148D464EB75E0C80144D492E0A92E00
:101D3000B12C23CE61E273E081010C511E4FC8012A
:101D400039D46CE973E0C80135D469EC75E0C80199
:101D500031D482E0A82EB12C60CE11821082F10124
:101D6000E251FE4F80819181009741F46EE573E06E
:101D700081010C511E4FC8011DD4BFC0019709F04D
:101D8000CCC00E94A6068C01FC0180819181A281B9
:101D9000B381181619061A061B0644F081E090E07C
:101DA000A0E0B0E080839183A283B383F8018481B3
:101DB0009581A681B781181619061A061B0644F0EC
:101DC00081E090E0A0E0B0E084839583A683B783B0
:101DD000F80180859185A285B385181619061A0623
:101DE0001B0644F081E090E0A0E0B0E0808791879E
:101DF000A287B387CE0101960E948B396EED74E005
:101E0000CE010196D7D360EF75E0CE010196D2D313
:101E100060914A0770914B0780914C0790914D0754
:101E20000E944A4C6B017C01D8016D917D918D918E
:101E30009C910E944A4C9B01AC01C701B6010E94D3
:101E4000384EAB01BC01CE0101960E945A3960E0C8
:101E500076E0CE010196AED360914E0770914F07A8
:101E600080915007909151070E944A4C6B017C0170
:101E7000F80164817581868197810E944A4C9B019B
:101E8000AC01C701B6010E94384EAB01BC01CE01C6
:101E900001960E945A3960E176E0CE0101968AD31C
:101EA00060915207709153078091540790915507A4
:101EB0000E944A4C6B017C01D80118966D917D916E
:101EC0008D919C911B970E944A4C9B01AC01C701CC
:101ED000B6010E94384EAB01BC01CE0101960E94B2
:101EE0005A39BE016F5F7F4F81010C511E4FC801EF
:101EF0006FD389819A810E946B470E94A606BC011C
:101F0000CE0101960E946C05BE016F5F7F4FC80134
:101F10005FD389819A810E946B47F101E251FE4FA4
:101F2000808191810196823091051CF49183808398
:101F300002C011821082F101E451FE4F1182108221
:101F40006CCA65962FAD6597211114CE20CE8CE119
:101F500095E00E945939C5010E94E93A8CE993E065
:101F60000E9459390E94A606B0924507A0924407E4
:101F7000C501EA960FB6F894DEBF0FBECDBFDF9164
:101F8000CF911F910F91FF90EF90DF90CF90BF9076
:101F9000AF909F908F907F906F905F904F903F9009
:101FA0002F900895CF92DF92EF92FF920F931F939D
:101FB000CF93DF936C017A018B01C0E0D0E0CE15A6
:101FC000DF0581F0D8016D918D01D601ED91FC9175
:101FD0000190F081E02DC6011995892B11F0219611
:101FE000EECF7E01C701DF91CF911F910F91FF903E
:101FF000EF90DF90CF900895089580E090E00895ED
:10200000FC01538D448D252F30E0842F90E0821BFE
:10201000930B541710F0CF96089501970895FC0183
:10202000918D828D981761F0828DDF01A80FB11D0F
:102030005D968C91928D9F5F9F73928F90E0089533
:102040008FEF9FEF0895FC01918D828D981731F0ED
:10205000828DE80FF11D858D90E008958FEF9FEF41
:102060000895FC01918D228D892F90E0805C9F4F17
:10207000821B91098F739927089587EF9BE0F1DF09
:1020800021E0892B09F420E0822F0895FC01848D42
:10209000DF01A80FB11DA35ABF4F2C91848D90E092
:1020A00001968F739927848FA689B7892C93A0896D
:1020B000B1898C91837080648C93938D848D9813F7
:1020C00006C00288F389E02D80818F7D808308958A
:1020D000EF92FF920F931F93CF93DF93EC0181E078
:1020E000888F9B8D8C8D981305C0E889F989808134
:1020F00085FD25C0F62E0B8D10E00F5F1F4F0F736F
:102100001127E02E8C8DE8120BC00FB607FCFACF1A
:10211000E889F989808185FFF5CFCE01B7DFF2CF5D
:102120008B8DFE01E80FF11DE35AFF4FF0829FB740
:10213000F8940B8FEA89FB89808180620AC09FB77F
:10214000F894EE89FF896083E889F989808183703A
:10215000806480839FBF81E090E0DF91CF911F91E9
:102160000F91FF90EF900895CF93DF93EC01888D4E
:102170008823C1F0EA89FB89808185FD05C0A88993
:10218000B9898C9186FD0EC00FB607FCF5CF808112
:1021900085FFF2CFA889B9898C9185FFEDCFCE015B
:1021A00075DFE8CFDF91CF91089580E090E0892B33
:1021B00019F063DF811125C080E090E0892B41F0A8
:1021C00080E090E0892B21F00E94000081111CC06A
:1021D00080E090E0892B41F080E090E0892B21F0B5
:1021E0000E940000811113C080E090E0892BA1F0D3
:1021F00080E090E0892B81F00E94000081110AC0EC
:1022000008950E940000D8CF0E940000E1CF0E94F4
:102210000000EACF0C94000008950F93FC01928512
:10222000908783858187A48DB58D119721F46217DE
:1022300021F0401711F06287438783858823D1F00E
:10224000828591110AC08823A9F080899189A28989
:10225000B3890197A109B10909C081110BC0808917
:102260009189A289B3890196A11DB11D808B918BA3
:10227000A28BB38B0F910895EBE0F1E08081877F13
:1022800080830895EBE0F1E0808188608083089589
:102290008E9808958E9A089514980895149A089522
:1022A00088980895889A08950E94D04FCF92DF921F
:1022B000EF92FF920F931F93CF93DF936C018B01EB
:1022C0007A01EC01C751D44F888187FF04C0FB011C
:1022D0001182108224C02CE02C9DC0012D9D900DF8
:1022E00011242881AC01420F511D27FD5A952091E0
:1022F0002C0D30E04217530794F42881AC01420FB3
:10230000511D27FD5A959A01FA01EE0FFF1F2E0F5E
:102310003F1FF901E456F34F208126FD19C0888143
:102320008F5F88832CE02C9DC0012D9D900D112482
:102330002881AC01420F511D27FD5A9520912C0D8B
:1023400030E042175307BCF428812C3044F113C00D
:102350002881820F911D27FD9A95FC01EE0FFF1F2A
:102360008E0F9F1FFC01E456F34F808160E08F7356
:102370000E94163BD4CFF80180819181049680346D
:102380009C4918F480E49CE904C0F80180819181A3
:102390000496F701918380838FEF888345C0F8010D
:1023A000408151812881BC01620F711D27FD7A9502
:1023B0009B01FB01EE0FFF1F2E0F3F1FF901E4569B
:1023C000F34F21813281240F351FF70131832083A0
:1023D0002881AC01420F511D27FD5A959A01FA013F
:1023E000EE0FFF1F2E0F3F1FF901E456F34F208120
:1023F00026FF1AC02881820F911D27FD9A95FC01A6
:10240000EE0FFF1F8E0F9F1FFC01E456F34F8081DC
:1024100061E08F73DF91CF911F910F91FF90EF904B
:10242000DF90CF900C94163BDF91CF911F910F91CD
:10243000FF90EF90DF90CF90089560E0FC018385DE
:102440000C94163B60E0FC0185810C94163B61E026
:10245000FC0183850C94163B61E0FC0185810C94A2
:10246000163B0F93CF93DF938091E80B81114AC005
:1024700081E08093E80B0E94AC24EC0106B126B108
:1024800040910001609100010295017026FB222716
:1024900020F941706695617082589E4FBEDE06B18C
:1024A00026B140B160B1017022FB222720F943FB25
:1024B000442740F966956170CE0180569E4FADDE8F
:1024C00002B322B340B160B1017022FB222720F990
:1024D000441F4427441F65FB662760F9CE018E53D5
:1024E0009E4F9BDECE0140960E94892DCE018657DD
:1024F0009F4F0E94892DCE018C5F9E4F0E94892D97
:102500001092E80BDF91CF910F9108950F931F93D5
:10251000CF93DF93EC0188819981009729F02A817C
:102520003B812617370788F48B016F5F7F4F0E942E
:10253000ED4E009761F0998388831B830A832C8179
:102540003D81232B11F4FC01108281E001C080E069
:10255000DF91CF911F910F910895EF92FF920F930A
:102560001F93CF93DF936115710511F480E01BC0B9
:1025700041155105B9F07B01EC018C819D818A01E7
:10258000080F191FB801CE01C1DF882379F3288114
:1025900039818C819D81B701820F931F0E94E64F84
:1025A0001D830C8381E0DF91CF911F910F91FF90EC
:1025B000EF9008956115710549F0FB01019000202D
:1025C000E9F73197AF01461B570BC7CF80E008955D
:1025D000FB014481558160817181BFCF1F920F92B1
:1025E0000FB60F9211240BB60F922F933F934F9378
:1025F0005F936F937F938F939F93AF93BF93EF936B
:10260000FF9387EF9BE042DDFF91EF91BF91AF9188
:102610009F918F917F916F915F914F913F912F91FA
:102620000F900BBE0F900FBE0F901F9018951F922A
:102630000F920FB60F9211240BB60F922F938F9318
:102640009F93EF93FF93E091070CF091080C80812A
:10265000E0910D0CF0910E0C82FD12C090818091E2
:10266000100C8F5F8F732091110C821751F0E09145
:10267000100CF0E0E950F44F958F8093100C01C0DE
:102680008081FF91EF919F918F912F910F900BBEC1
:102690000F900FBE0F901F901895CF92DF92EF9280
:1026A000FF92CF93DF93EC01603282E078070CF069
:1026B0003DC077FD06C0653B71052CF064EB70E012
:1026C00002C060E070E0898128E830E06901C81A42
:1026D000D10887FDD394CC0CDD1CCC0CDD1C0D2C5B
:1026E000000CEE08FF088A8128E532E0281B31093A
:1026F00087FD3395220F331F220F331FC901330F7C
:10270000AA0BBB0B9C01AD012C193D094E095F09B9
:10271000DB010E949C4D24EB30E040E050E00E9441
:10272000764DC20ED31EE41EF51EB601388130333D
:1027300080F5298188E890E0821B910927FD939517
:10274000880F991F880F991F6817790784F08A816D
:1027500048E552E0481B510987FD5395440F551F2A
:10276000440F551FCB01461757070CF4CA010297B7
:10277000880F991F4FB7F894232F30E0F901EE0F1F
:10278000FF1F2E0F3F1FF901E456F34F9283818301
:102790004FBFDF91CF91FF90EF90DF90CF900895E2
:1027A0001F93CF93DF93EC01162F8881803308F0BD
:1027B0004EC061E0812F0E94443B8881E82FF0E009
:1027C0009F01220F331FE20FF31FE456F34F1F73D5
:1027D0009081907C192B108319821A826CE00E94E0
:1027E000D94E9CE0899FB001112440E050E09B014C
:1027F000240F351FF901EE0FFF1F2E0F3F1FF901A8
:10280000E456F34F908196FD16C04F5F5F4F4C30FA
:10281000510569F7813001F51092800082E08093C4
:1028200081001092850010928400B19A80916F000F
:10283000826080936F00E881F0E0CF01880F991FDC
:10284000E80FF91FE456F34F80818064808388810C
:10285000DF91CF911F910895823061F41092900022
:1028600080939100109295001092940088BB809301
:102870007100E1CF833069F41092A00082E0809370
:10288000A1001092A5001092A40089BB8093720051
:10289000D2CF8111D0CF1092200182E0809321010C
:1028A00010922501109224018ABB80937300C3CF3C
:1028B0001F920F920FB60F9211240BB60F922F9307
:1028C0003F934F935F936F937F938F939F93AF93B8
:1028D000BF93EF93FF9348E251E064E271E080E040
:1028E00090E0E4DCFF91EF91BF91AF919F918F91C8
:1028F0007F916F915F914F913F912F910F900BBE00
:102900000F900FBE0F901F9018951F920F920FB649
:102910000F9211240BB60F922F933F934F935F9317
:102920006F937F938F939F93AF93BF93EF93FF9397
:1029300048EA50E064EA70E083E090E0B7DCFF91A1
:10294000EF91BF91AF919F918F917F916F915F9127
:102950004F913F912F910F900BBE0F900FBE0F9094
:102960001F9018951F920F920FB60F9211240BB65D
:102970000F922F933F934F935F936F937F938F9318
:102980009F93AF93BF93EF93FF9348E950E064E9BF
:1029900070E082E090E08ADCFF91EF91BF91AF910F
:1029A0009F918F917F916F915F914F913F912F9167
:1029B0000F900BBE0F900FBE0F901F9018951F9297
:1029C0000F920FB60F9211240BB60F922F933F93D5
:1029D0004F935F936F937F938F939F93AF93BF9327
:1029E000EF93FF9348E850E064E870E081E090E006
:1029F0005DDCFF91EF91BF91AF919F918F917F919E
:102A00006F915F914F913F912F910F900BBE0F905F
:102A10000FBE0F901F9018951F920F920FB60F9236
:102A200011240BB60F922F933F934F935F936F93A5
:102A30007F938F939F93AF93BF93EF93FF93E09117
:102A40004207F09143071995FF91EF91BF91AF9124
:102A50009F918F917F916F915F914F913F912F91B6
:102A60000F900BBE0F900FBE0F901F901895CF9335
:102A7000DF93EC0188810E94EE3A21E0892B09F472
:102A800020E02C878C810E94EE3A21E0892B09F40A
:102A900020E02E878C8D9D8D0197D1F48A810E9434
:102AA000EE3A21E0892B09F420E02D878E810E94E7
:102AB000EE3A21E0892B09F420E02F879C858D8553
:102AC000981749F08E85281731F09A878B8703C0B5
:102AD0008C858A872B87DF91CF910895CF92DF92E3
:102AE000EF92FF920F931F93CF93DF93FC016489C2
:102AF000758986899789C68DD78D603127E27207DF
:102B00008105910529F0161617061806190644F0D6
:102B10002089318942895389DE010E949C4D2AC057
:102B20008F010E944A4C20E030E44CE156E40E94C0
:102B3000384E6B017C01F801608F718F828F938F0B
:102B400060897189828993890E944A4CA701960104
:102B50000E94A94C6B017C01BE01DD0F880B990B13
:102B60000E944A4C9B01AC01C701B6010E94A94CCE
:102B70000E94A04EDF91CF911F910F91FF90EF9097
:102B8000DF90CF900895FC0181E090E091A380A3B5
:102B90001182108215821482108A118A128A138A75
:102BA000158E148E80E197E2A0E0B0E0848B958BC7
:102BB000A68BB78B12861086148615861686178606
:102BC0000895CF93DF93EC01FC01E759FF4F10828A
:102BD000379781E0808360E08D810E94163B8F856E
:102BE0009889892B31F060E08B85DF91CF910C942F
:102BF000163BDF91CF910895CF93DF93EC018B8942
:102C00000E94EE3A2E8930E08217930711F48F89E3
:102C100001C080E0DF91CF910895CF93DF93EC0165
:102C200089890E94EE3A2E8930E08217930711F4C9
:102C30008F8901C080E0DF91CF910895CF93DF931A
:102C4000EC018DA5882311F061E001C060E08F8167
:102C50000E94163B8EA5882329F08FA5882311F0AA
:102C600061E001C060E08D85DF91CF910C94163B4F
:102C7000CF93DF93EC018DA5882311F060E001C0B4
:102C800061E08F810E94163B8EA5882329F08FA5D5
:102C9000882311F060E001C061E08D85DF91CF9164
:102CA0000C94163BCF93DF93EC0161E089850E9481
:102CB000163B8EA5882321F061E08F850E94163B8C
:102CC000C959DF4F1882DF91CF910895CF93DF93D9
:102CD000EC0160E089850E94163B8EA5882321F0D7
:102CE00060E08F850E94163BC959DF4F81E08883E1
:102CF000DF91CF910895CF92DF92EF92FF920F93E1
:102D00001F93CF93DF93FC0142AF53AF64AF75AF16
:102D1000DC01DE964D935D936D937C93139714962F
:102D20000D931D932D933C931397EC01CA5BDF4FDA
:102D3000E88284A9882389F084A5811109C037FF1E
:102D40000CC01D921D921D921C92139781E006C02B
:102D50001016110612061306A4F380E045A956A921
:102D600067A970AD14161506160617063CF591AD49
:102D7000992321F10D911D912D913C91139768019B
:102D8000790137FF07C0CC24DD247601C01AD10AAF
:102D9000E20AF30A4C155D056E057F057CF437FFEA
:102DA00007C070956095509541955F4F6F4F7F4F6D
:102DB0004D935D936D937C93139781E0DF01A15B4D
:102DC000BF4F1D921D921D921C921397E15AFF4F07
:102DD00091E09083DF91CF911F910F91FF90EF9041
:102DE000DF90CF9008950F931F93CF93DF938C01C3
:102DF000D62FFC018589811109C0C8010EDFC82FBB
:102E0000C801FADED11108C08C2F06C0C801F4DE5B
:102E1000C82FC80102DFF6CFDF91CF911F910F912C
:102E20000895CF93DF93EC01FC01E759FF4F81E058
:102E3000808339978081B297882341F08081918186
:102E4000A281B3810196A11DB11D07C0808191812E
:102E5000A281B3810197A109B10980839183A283E3
:102E6000B383FE01E459FF4F20813181DE01A65971
:102E7000BF4FC9019595879520FD03C0ED91FC9149
:102E80000DC0FE01E80FF91F0190F081E02D2D919A
:102E90003C91E20FF31F0190F081E02D8C0F9D1FFC
:102EA00019958F859889892B11F1FE01E059FF4F03
:102EB00020813181DE01A259BF4FC90195958795C7
:102EC00020FD03C0ED91FC910DC0FE01E80FF91F3C
:102ED0000190F081E02D2D913C91E20FF31F0190C4
:102EE000F081E02D8C0F9D1FDF91CF911994DF9120
:102EF000CF9108958F929F92AF92BF92CF92DF921F
:102F0000EF92FF920F931F93CF93DF93EC01FC019D
:102F1000E15BFF4F60817181828193810E94484C07
:102F20006B017C0168A979A98AA99BA90E944A4CD6
:102F30009B01AC0160E074E284E799E40E94384EA2
:102F40004B015C01FE01E55AFF4F60817181828176
:102F500093810E94484C9B01AC01C501B4010E94C1
:102F6000384E4B015C018E010D5A1F4F20E030E0BE
:102F700040E05FE30E94A94CA70196010E94D44D56
:102F80000E94A54EF8016083718382839383C95A9E
:102F9000DF4FA5019401C701B6010E94D44D0E94E4
:102FA000A54E688379838A839B83DF91CF911F919C
:102FB0000F91FF90EF90DF90CF90BF90AF909F90D8
:102FC0008F900895603E710508F0D8C3FB018827F3
:102FD000EE58FF4F8F4F0C94E54E81E090E0A0E05B
:102FE000B0E08093560790935707A0935807B0938B
:102FF0005907089510925A0710925B0710925C07C8
:1030000010925D07089510925E0710925F0710926C
:10301000600710926107089581E090E0A0E0B0E0C1
:103020008093620790936307A0936407B09365074A
:103030000895109266071092670710926807109221
:103040006907089583E090E0A0E0B0E080936A070C
:1030500090936B07A0936C07B0936D07089588E772
:1030600090E0A0E0B0E08093820790938307A09364
:103070008407B0938507089588E790E0A0E0B0E06A
:103080008093860790938707A0938807B09389075A
:10309000089588E790E0A0E0B0E080938A079093DD
:1030A0008B07A0938C07B0938D0708951092920719
:1030B000109293071092940710929507089510921A
:1030C0009607109297071092980710929907089503
:1030D00081E090E0A0E0B0E080939A0790939B0796
:1030E000A0939C07B0939D07089510929E0710929D
:1030F0009F071092A0071092A10708951092A207AF
:103100001092A3071092A4071092A5070895109299
:10311000A6071092A7071092A8071092A907089572
:103120001092AA071092AB071092AC071092AD074D
:1031300008951092AE071092AF071092B007109248
:10314000B10708951092B2071092B3071092B40716
:103150001092B50708951092BA071092BB0710920B
:10316000BC071092BD0708951092BE071092BF07CA
:103170001092C0071092C10708951092C2071092D2
:10318000C3071092C4071092C50708951092D20782
:103190001092D3071092D4071092D5070895109279
:1031A000D6071092D7071092D8071092D907089522
:1031B0001092DA071092DB071092DC071092DD07FD
:1031C000089581E090E0A0E0B0E08093E60790935E
:1031D000E707A093E807B093E907089581E090E03E
:1031E000A0E0B0E08093EA079093EB07A093EC0790
:1031F000B093ED0708958CE291E0A0E0B0E08093F9
:10320000FA079093FB07A093FC07B093FD0708957E
:103210008CE291E0A0E0B0E08093FE079093FF077E
:10322000A0930008B093010808958CE291E0A0E01B
:10323000B0E08093020890930308A0930408B09331
:103240000508089510920A0810920B0810920C08B5
:1032500010920D08089510920E0810920F08109207
:103260001008109211080895109212081092130875
:1032700010921408109215080895109222081092C6
:103280002308109224081092250808951092260809
:10329000109227081092280810922908089581E0BA
:1032A00090E0A0E0B0E080932A0890932B08A093D0
:1032B0002C08B0932D08089585E090E0A0E0B0E0E0
:1032C0008093320890933308A0933408B093350864
:1032D000089585E090E0A0E0B0E0809336089093F8
:1032E0003708A0933808B0933908089589E190E031
:1032F000A0E0B0E080933A0890933B08A0933C088C
:10330000B0933D08089582E390E0A0E0B0E08093A0
:103310004A0890934B08A0934C08B0934D08089529
:1033200082E390E0A0E0B0E080934E0890934F08D5
:10333000A0935008B0935108089582E390E0A0E074
:10334000B0E08093520890935308A0935408B09330
:103350005508089582E390E0A0E0B0E080935A0819
:1033600090935B08A0935C08B0935D08089582E396
:1033700090E0A0E0B0E080935E0890935F08A09397
:103380006008B0936108089582E390E0A0E0B0E0A7
:103390008093620890936308A0936408B0936508D3
:1033A000089580E991E0A0E0B0E0809372089093E6
:1033B0007308A0937408B0937508089580E991E0AC
:1033C000A0E0B0E08093760890937708A093780807
:1033D000B0937908089580E991E0A0E0B0E080938F
:1033E0007A0890937B08A0937C08B0937D08089599
:1033F0001092820810928308109284081092850817
:1034000008951092860810928708109288081092EA
:103410008908089510928A0810928B0810928C08DF
:1034200010928D08089510929A0910929B0910929B
:103430009C0910929D09089510929E0910929F096F
:103440001092A0091092A10908951092A209109259
:10345000A3091092A4091092A50908951092EA08F0
:103460001092EB081092EC081092ED08089510925B
:10347000EE081092EF081092F0081092F1080895EB
:103480001092F2081092F3081092F4081092F508C6
:1034900008951092FA081092FB081092FC081092FE
:1034A000FD0808951092FE081092FF08109200097E
:1034B00010920109089510920209109203091092C6
:1034C000040910920509089585E090E0A0E0B0E0BD
:1034D0008093120990931309A0931409B0931509CE
:1034E000089585E090E0A0E0B0E080931609909305
:1034F0001709A0931809B0931909089585E090E081
:10350000A0E0B0E080931A0990931B09A0931C09D6
:10351000B0931D09089584EB95E1A0E0B0E080939D
:10352000220990932309A0932409B09325090895B3
:1035300084EB95E1A0E0B0E0809326099093270901
:10354000A0932809B0932909089584EB95E1A0E0A0
:10355000B0E080932A0990932B09A0932C09B09393
:103560002D09089585E090E0A0E0B0E080933A094D
:1035700090933B09A0933C09B0933D09089585E0E1
:1035800090E0A0E0B0E080933E0990933F09A093C3
:103590004009B0934109089585E090E0A0E0B0E0D3
:1035A0008093420990934309A0934409B09345093D
:1035B000089510924A0910924B0910924C091092EA
:1035C0004D09089510924E0910924F09109250091A
:1035D00010925109089510925209109253091092B5
:1035E00054091092550908951092620910926309C6
:1035F000109264091092650908951092660910925C
:1036000067091092680910926909089510926A0971
:1036100010926B0910926C0910926D090895109226
:103620007A0A10927B0A10927C0A10927D0A089501
:103630008CE390E0A0E0B0E080937E0A90937F0A54
:10364000A093800AB093810A089581E090E0A0E001
:10365000B0E08093820A9093830AA093840AB09387
:10366000850A089510928A0A10928B0A10928C0A89
:1036700010928D0A08958CE390E0A0E0B0E0809372
:103680008E0A90938F0AA093900AB093910A08959E
:1036900081E090E0A0E0B0E08093920A9093930ADA
:1036A000A093940AB093950A08951092A20A1092DA
:1036B000A30A1092A40A1092A50A08958CE390E040
:1036C000A0E0B0E08093A60A9093A70AA093A80A6E
:1036D000B093A90A089581E090E0A0E0B0E0809363
:1036E000AA0A9093AB0AA093AC0AB093AD0A0895CE
:1036F0001092B20A1092B30A1092B40A1092B50A4C
:1037000008958CE390E0A0E0B0E08093B60A909337
:10371000B70AA093B80AB093B90A089581E090E07F
:10372000A0E0B0E08093BA0A9093BB0AA093BC0AD1
:10373000B093BD0A08951092CA0A1092CB0A109253
:10374000CC0A1092CD0A08958CE390E0A0E0B0E09E
:103750008093CE0A9093CF0AA093D00AB093D10A57
:10376000089581E090E0A0E0B0E08093D20A9093C9
:10377000D30AA093D40AB093D50A0895660F771F91
:10378000660F771FFB01EA5AF84F108211821282EE
:10379000138208958FEF9FEF08954F925F926F927B
:1037A0007F928F929F92AF92BF92CF92DF92EF92D1
:1037B000FF920F931F93CF93DF938B01EB01CC0FFD
:1037C000DD1FCE010E94604D882E912CA12CB12CC2
:1037D000CE0101960E94604DC82ED12CE12CF12C17
:1037E0000D5811090330110588F5CE0144960E9449
:1037F000604D482E512C612C712CCE0145960E94B3
:10380000604D482F50E060E070E08FEF48165104A3
:1038100061047104A9F44F3F51056105710581F4FC
:103820008FEF88169104A104B10481F48FEFC816BC
:10383000D104E104F10451F46FEF7FEFCB012BC011
:1038400040385105610571056CF0F6CF80E8C81667
:10385000D104E104F10484F740E050E0BA01412CC6
:10386000512C3201FE2CED2CDC2CCC248C0C9D1C1C
:10387000AE1CBF1C320155244424840C951CA61C8C
:10388000B71C742F662755274427CB01BA01680D52
:10389000791D8A1D9B1DDF91CF911F910F91FF9084
:1038A000EF90DF90CF90BF90AF909F908F907F90E0
:1038B0006F905F904F9008958EED95E00E9459397A
:1038C00089E393E00E9459390E94A6060E94B00540
:1038D00080E090E008950C946B470C946B470C9437
:1038E0006B470C946B470C946B470C946B474F924F
:1038F0005F926F927F928F929F92AF92BF92CF9280
:10390000DF92EF92FF920F931F93CF93DF9300D03C
:1039100000D0CDB7DEB7FB0126892D8387898E8342
:1039200082889388A684B784C284D384E484F5848F
:10393000468057806084718482819381A481B5819F
:1039400089839A83AB83BC830E94AC241F921F920D
:103950001F92AE81AF93BD81BF93930182014981D4
:103960005A816B817C810E9480070F900F900F908D
:103970000F900F9080E090E026960FB6F894DEBF8F
:103980000FBECDBFDF91CF911F910F91FF90EF90B0
:10399000DF90CF90BF90AF909F908F907F906F906F
:1039A0005F904F900895CF93DF93EB0120E030E0DC
:1039B00040E85FE36A817B818C819D810E94444C59
:1039C000811112C083EE95E00E945939C5D7FC01E0
:1039D000E25BFF4F1082118212821382E05DFE4F84
:1039E000108A118A128A138A20E030E040E85FE3EF
:1039F0006E817F81888599850E94444C811112C017
:103A000083EF95E00E945939A7D7FC01E853FF4F97
:103A10001082118212821382E852FF4F108A118A9B
:103A2000128A138A20E030E040E85FE36A857B85F4
:103A30008C859D850E94444C811112C083E096E0E4
:103A40000E94593989D7FC01EE5BFE4F108211822A
:103A500012821382E058FF4F108A118A128A138A49
:103A60000E94A6060E94B00580E090E0DF91CF9111
:103A700008956E3471050CF050C06B3471050CF074
:103A80008FC06C32710554F5693271050CF088C035
:103A90006831710594F46F3071050CF081C06630A7
:103AA000710544F4623071050CF07AC0672B09F09F
:103AB00075C076C06B5071096EC0623271053CF4FE
:103AC0006F3171050CF06CC06951710964C06452AA
:103AD00071096230710508F061C062C06A33710516
:103AE0007CF4673371050CF05BC06D3271050CF42A
:103AF00055C0603371050CF453C0635371094BC05A
:103B0000643471053CF4613471050CF049C06D53A7
:103B1000710941C0675471093EC066387105F4F4FB
:103B200063387105ECF56237710564F46F36710521
:103B3000BCF56536710594F1683671058CF16956EE
:103B4000710929C06C37710534F46937710544F582
:103B50006357710920C06D5771091DC0603D710523
:103B60007CF46D3C7105E4F46439710534F4613919
:103B70007105B4F46D5871090EC0695C71090BC010
:103B80006A3D710534F4673D710554F4635D710954
:103B900002C06D5D71096330710510F080E0089519
:103BA00081E008950F931F93CF93DF938C01C0E0C2
:103BB000D0E0BE01C8015DDF882319F0BE01C80155
:103BC00001DA2196C13ED105A1F7DF91CF911F9176
:103BD0000F910895CF92DF92EF92FF920F931F9370
:103BE000CF93DF938B0169017A01EB01CC0FDD1FCD
:103BF0006C2DCE010E94684D9927F7FC9A958F2D68
:103C00007E2D6D2DCE0101960E94684D0D58110933
:103C10000330110588F4B701992777FD9095892F16
:103C2000CE0144960E94684D6F2D772788279927EB
:103C3000CE0145960E94684D80E090E0DF91CF91E3
:103C40001F910F91FF90EF90DF90CF900895CF924A
:103C5000DF92EF92FF92CF93DF93EB010ADF88238D
:103C600059F1FE01EE0FFF1FEE0FFF1FEA5AF84F4A
:103C7000C080D180E280F38083E196E00E945939D0
:103C800081EE95E00E94593987E196E00E9459390A
:103C9000CE010E94E93A81EE95E00E94593989E10E
:103CA00096E00E945939C701B6010E94F9390E9475
:103CB000A6060E94B00504C08DE994E00E9459391F
:103CC00080E090E0DF91CF91FF90EF90DF90CF9078
:103CD0000895EF92FF920F931F93CF93DF938091FC
:103CE000ED0B9091EE0B892B09F064C084E090E01D
:103CF0000E94D346EC0160E070E04FDD1616170617
:103D0000F4F0CE014FDF96E5E92E97E0F92E00E0C2
:103D100010E0B801CE01ADDE882341F0F70120812B
:103D2000318142815381B801CE0154DF0F5F1F4FB3
:103D3000F4E0EF0EF11C0639110559F737C063E0C6
:103D400070E0CE012ADD613071058105910561F5D4
:103D500086E5E82E87E0F82E00E010E0B801CE01FD
:103D600088DE8823C1F0B801CE0117DDF70160833A
:103D70007183828393836F3F7F4F8F4F9F4F59F49F
:103D8000B801CE011FD9F7012081318142815381D1
:103D9000B801CE011FDF0F5F1F4FF4E0EF0EF11CE3
:103DA000013E1105D9F602C0CE01FCDED093EE0B28
:103DB000C093ED0B8091ED0B9091EE0BDF91CF91C5
:103DC0001F910F91FF90EF9008954F925F926F9225
:103DD0007F928F929F92AF92BF92CF92DF92EF929B
:103DE000FF920F931F93CF93DF9300D01F92CDB715
:103DF000DEB76FDF4090320850903308609034088F
:103E00007090350866DF8090360890903708A09053
:103E10003808B09039080E94A606C0904A07D09092
:103E20004B07E0904C07F0904D070E94A606C70193
:103E3000B6010E944A4C6B017C01C301B2010E9491
:103E40004A4C9B01AC01C701B6010E94384E2B01C0
:103E50003C0160914E0770914F07809150079091FF
:103E600051070E944A4C6B017C01C501B4010E94BC
:103E70004A4C9B01AC01C701B6010E94384E6983D0
:103E80007A838B839C8368D51F921F921F921F9207
:103E90001F92812C912CA12CB12CC12CD12C7601FC
:103EA00009811A812B813C81B301A2010E94800704
:103EB00053D51F921F921F921F921F929701860146
:103EC000B301A2010E94800747D51F921F921F9243
:103ED0001F921F9297018601B701A6010E948007D9
:103EE0000FB6F894DEBF0FBECDBF80E090E00F901C
:103EF0000F900F900F90DF91CF911F910F91FF9036
:103F0000EF90DF90CF90BF90AF909F908F907F9079
:103F10006F905F904F9008950895089508950895C3
:103F200008950895CF92DF92EF92FF920F931F931F
:103F3000CF93DF937C016B018A01E901CADEF601B0
:103F4000EE0FFF1FEE0FFF1FEA5AF84F808191819D
:103F5000F70191838083BDDE000F111F000F111F39
:103F6000F801EA5AF84F81E0408151816281738102
:103F7000413051056105710509F080E0F701828744
:103F8000A8DECC0FDD1FCC0FDD1FCA5AD84F8881A9
:103F90009981AA81BB81F70182839383A483B5832E
:103FA0001682178210861186DF91CF911F910F9193
:103FB000FF90EF90DF90CF900895AF92BF92CF9295
:103FC000DF92EF92FF920F931F93CF93DF93EC0159
:103FD00086E390E09E8B8D8B87E390E0988F8F8BAC
:103FE00086E290E09A8F898F8AE190E09C8F8B8F98
:103FF0008CE190E09E8F8D8F88E190E098A38F8F69
:1040000083E090E09AA389A382E090E09CA38BA335
:10401000FE01E657FF4F8CE390E0968385838DE3A6
:1040200090E09087878388E390E092878187148669
:10403000138616861586108A17868EE090E0928B7E
:10404000818B8FE090E0948B838BE658FF4F8EE25C
:1040500090E09683858380E390E0908787838EE36A
:1040600090E0928781871486138616861586108ABB
:10407000178682E190E0928B818B83E190E0948BB4
:10408000838BEF50FF4F1182108232961182108283
:10409000329611821082CE01A0D6CE010E94BF318D
:1040A0006E0182E8C81A8EEFD80AAA24A394B12C14
:1040B000F601B1A2A0A27E01F0E6EF1AFEEFFF0A20
:1040C00084E090E0F70191A380A38E010E531E4F70
:1040D00088E090E0F80191A380A380E190E0F601F0
:1040E0009183808381E190E0958384838FE190E0E8
:1040F0009383828381E290E097838683C6010E9446
:104100003715F601828580878385818787E190E076
:10411000F7019183808389E190E09583848383E232
:1041200090E09383828385E290E097838683C70142
:104130000E943715F70182858087838581878BE10F
:1041400090E0F801918380838DE190E095838483F2
:1041500087E290E09383828389E290E0978386836D
:10416000C8010E943715F801828580878385818781
:10417000E25FFE4F8081918172974081518162811F
:104180007381369720813181F601358F248F448BDE
:10419000558B668B778B019729F48FEF9FEF978F65
:1041A000868F03C0F601B78EA68EFE01EE52FD4F3C
:1041B00080819181709740815181628173813897AC
:1041C00020813181F701358F248F448B558B668B8D
:1041D000778B019719F48FEF9FEF03C081E090E098
:1041E000F701978F868FFE01EC52FD4F8081918100
:1041F0003E974081518162817381C454DD4F288193
:104200003981F801358F248F448B558B668B778BE2
:10421000019719F48FEF9FEF03C081E090E0F80160
:10422000978F868FDF91CF911F910F91FF90EF9025
:10423000DF90CF90BF90AF9008952F923F924F9212
:104240005F926F927F928F929F92AF92BF92CF9226
:10425000DF92EF92FF920F931F93CF93DF93CDB72F
:10426000DEB7CA57D1090FB6F894DEBF0FBECDBF77
:104270008C01FC0110821182128213821482158239
:10428000168217821086118612861386148615866A
:10429000168617864C01F0E18F0E911CC4010E9416
:1042A000673068018AE8C80ED11CC6010E946730D9
:1042B0007801ECEFEE1AEEEFFE0AC7010E946730BC
:1042C0005801F2E8AF1AFEEFBF0AC5010E94C315FC
:1042D000380180E6681A8EEF780AC3010E94C31580
:1042E0002801EEE34E1AEEEF5E0AC2010E94C315EA
:1042F000C8018C519E4F0E948B39F801E651FE4F48
:1043000011821082329611821082329611821082AE
:104310003296118210823296108231961082319636
:10432000108231961182108232961182108232965A
:10433000118210823296108231961082319610824C
:104340003196108211821282138234961082118269
:104350001282138234961082118212821382349652
:10436000108211821282138234961082118212827C
:104370001382349610821182128213823496108234
:104380001182128213823496108211821282138259
:104390003496108211821282138234961082118216
:1043A0001282138234961082118212821382349602
:1043B000108211821282138234961082118212822C
:1043C00013823496108211821282138234961082E4
:1043D00011821282138234961082319610823196A5
:1043E00010823196108211821282138234961082CA
:1043F00011821282138234961082118212821382E9
:104400003496108231961082319610823196108245
:104410003196108231961082319610823196108238
:104420003196108231961082319610823196108228
:104430003196108231961082319610823196108218
:104440003196108231961082319610823196108208
:1044500031961082319610823196108231961082F8
:104460003196108211821282138234961082118248
:104470001282138234961082118212821382D80122
:10448000A359BD4F8CE0E2E4F3E001900D928A95D0
:10449000E1F7F801E758FD4F108211821282138272
:1044A0003496108211821282138234961082118205
:1044B00012821382349611821082329611821082F7
:1044C00032961182108232961082118212821382E9
:1044D00034961082118212821382349610821182D5
:1044E00012821382349610821182128213823496C1
:1044F00010821182128213823496108211821282EB
:104500001382349611821082329611821082329672
:104510001182108232961082118212821382349696
:1045200010821182128213823496108211821282BA
:104530001382349610823196108231961082319611
:10454000118210823296118210823296118210826C
:104550003296108211821282138234961082118256
:104560001282138234961082118212821382349640
:10457000118210823296118210823296118210823C
:1045800032961182108232961182108232961182F6
:104590001082329611821082329611821082180196
:1045A000F6E22F1AFDEF3F0AF1011082CE010196CB
:1045B0000E9467308AE7FE013196D40101900D9286
:1045C0008A95E1F7CE0101960E9467308AE7FE01E5
:1045D0003196D60101900D928A95E1F7CE010196B0
:1045E0000E9467308AE7FE013196D70101900D9253
:1045F0008A95E1F788E5F801808B89E5F6018083EB
:104600008AE5F7018083CE0101960E94C31582E2FC
:10461000FE013196D50101900D928A95E1F7CE0108
:1046200001960E94C31582E2FE013196D3010190EA
:104630000D928A95E1F7CE0101960E94C31582E2A0
:10464000FE013196D20101900D928A95E1F7C801E1
:10465000B4DCF1011082C658DF4F0FB6F894DEBF0C
:104660000FBECDBFDF91CF911F910F91FF90EF90C3
:10467000DF90CF90BF90AF909F908F907F906F9082
:104680005F904F903F902F9008950F931F93CF937B
:10469000DF938B01EA018AE593E00E94593981EEAC
:1046A00095E00E945939F80180810E94F439CE01C9
:1046B0000E94E93A0E94A606DF91CF911F910F91C7
:1046C0000C94B005CF92DF92EF92FF920F931F935D
:1046D000CF93DF93CDB7DEB728970FB6F894DEBF40
:1046E0000FBECDBF8B016A018C519E4F7C0166E5E8
:1046F00073E00E94DA1261EE75E0C7010E94DA12DF
:10470000F801808189831A8241E050E08E010F5FB9
:104710001F4FB801C7010E94AD124AE0B801C6019F
:104720000E942148F80101900020E9F73197AF017C
:10473000401B510BB801C7010E94AD120E94A60692
:10474000BC01C8010E946C05B801C7010E94E812B3
:1047500089819A810E946B4728960FB6F894DEBF34
:104760000FBECDBFDF91CF911F910F91FF90EF90C2
:10477000DF90CF900895FC01DB01AD59BF4F8C91C4
:10478000882319F022E030E002C020E030E0DB01B5
:10479000AB59BF4F8C91882311F023E030E0DB014F
:1047A000AC59BF4F8C91882311F024E030E0DB013D
:1047B000AA59BF4F8C91882311F026E030E0DA012E
:1047C0008D919C912817390721F091E0121613065C
:1047D0000CF090E0DA012D933C93992319F0A90194
:1047E000CF0170CF08958F929F92AF92BF92CF92D8
:1047F000DF92EF92FF920F931F93CF93DF93EC0121
:1048000082E593E00E94593980EF95E00E94593982
:104810006E0182E8C81A8EEFD80AC6010E946E1592
:104820000E944A4C4B015C01FE01E359FD4F60813F
:104830007181828193810E944A4C9B01AC01C50128
:10484000B4010E94384E42E00E94203A80E096E097
:104850000E9459397E01E0E6EE1AEEEFFE0AC7012A
:104860000E946E150E944A4C4B015C01FE01EF58FC
:10487000FD4F60817181828193810E944A4C9B012E
:10488000AC01C501B4010E94384E42E00E94203ABA
:1048900080E196E00E9459398E010E531E4FC801E7
:1048A0000E946E150E944A4C4B015C01CB58DD4FB3
:1048B000688179818A819B810E944A4C9B01AC016D
:1048C000C501B4010E94384E42E00E94203A0E9485
:1048D000A6060E94B0058EE493E00E94593980EF4D
:1048E00095E00E945939F601A68DB78D208931894E
:1048F000428953890E949C4D0E94F93980E096E0DC
:104900000E945939F701A68DB78D208931894289D6
:1049100053890E949C4D0E94F93980E196E00E94E3
:104920005939F801A68DB78D20893189428953897B
:104930000E949C4D0E94F9390E94A606DF91CF91FA
:104940001F910F91FF90EF90DF90CF90BF90AF90AD
:104950009F908F900C94B005CF93DF938091F50BCF
:104960009091F60B892B51F48BED92E00E94D34687
:10497000EC0163DCD093F60BC093F50B8091F50B43
:104980009091F60BDF91CF9108958091F30B909168
:10499000F40B892B41F481E090E00E94D346909380
:1049A000F40B8093F30B8091F30B9091F40B08952B
:1049B000CF93DF93EC012AEC30E04BEC50E069EC54
:1049C00070E0B0DA2EEC30E04FEC50E06DEC70E0CF
:1049D000CE010C96A7DA24ED30E045ED50E063ED12
:1049E00070E0CE0148969EDA28ED30E049ED50E0C7
:1049F00067ED70E0CE01849695DA2EED30E04FED54
:104A000050E06DED70E0CE01C096DF91CF918ACA83
:104A1000CF93DF938091F10B9091F20B892BE9F406
:104A20008CE390E00E94D346EC01FC01CC9611820D
:104A300010823C96E817F907D1F7198218821D8673
:104A40001C86198E188E1DA21CA219AA18AACE01A6
:104A5000AFDFD093F20BC093F10B8091F10B9091EB
:104A6000F20BDF91CF910895EF92FF920F931F9376
:104A7000CF93DF93162F072F7A014115510559F473
:104A8000862F0E94EE3A31E020E0019709F030E0F5
:104A9000C32FD22F26C04130510509F5862F66332A
:104AA00010F08AEC860F90917B00282F2870977F5A
:104AB000922B90937B008770806480937C00809120
:104AC0007A00806480937A0080917A0086FDFCCF22
:104AD000C091780080917900D0E0D82B02C0C0E06E
:104AE000D0E082E0E816F10410F58BE196E00E9438
:104AF000593981EE95E00E94593987E196E00E948C
:104B00005939812F902F0E94E93A81EE95E00E9459
:104B1000593989E196E00E945939CE010E94E93A5B
:104B20000E94A6060E94B00580E090E002C081E0ED
:104B300090E0DF91CF911F910F91FF90EF9008953A
:104B40000F931F93CF93DF93FB013197F49708F0F6
:104B5000D7C02230310508F0D3C0EA018B01FC0137
:104B600088E3829FA001839F500D1124E40FF51F5D
:104B7000E60FF71F81E08083232B11F46C2F07C011
:104B800061E0802F0E94443B209739F460E0802F41
:104B90000E94163B80E090E0B5C0CF3FD10509F4FC
:104BA000ADC0F801E550FB4FE4918E2F90E0FC0181
:104BB0003197E231F10508F09DC08827EE5AFE4F8B
:104BC0008F4F0C94E54E84B5806884BDC7BDE2CF9D
:104BD00084B5806284BDC8BDDDCF809180008068CF
:104BE00080938000D0938900C0938800D3CF8091B8
:104BF0008000806280938000D0938B00C0938A00F5
:104C0000C9CF80918000886080938000D0938D0010
:104C1000C0938C00BFCF8091B00080688093B000BB
:104C2000C093B300B7CF8091B00080628093B00092
:104C3000C093B400AFCF80919000806880939000C3
:104C4000D0939900C0939800A5CF80919000806286
:104C500080939000D0939B00C0939A009BCF80914B
:104C60009000886080939000D0939D00C0939C003A
:104C700091CF8091A00080688093A0008091A000D7
:104C80008F7B8093A000D093A900C093A80082CF0F
:104C90008091A00080628093A000D093AB00C0936D
:104CA000AA0078CF8091A00088608093A000D09364
:104CB000AD00C093AC006ECF8091200180688093DE
:104CC0002001D0932901C093280164CF8091200155
:104CD000806280932001D0932B01C0932A015ACF88
:104CE00080912001886080932001D0932D01C09392
:104CF0002C0150CFC038D1050CF448CF61E047CF2C
:104D000081E090E0DF91CF911F910F910895809104
:104D1000EF0B9091F00B892B91F480E790E00E94CB
:104D2000D346FC0131969C012B5C3F4F119217AA90
:104D3000E217F307D9F79093F00B8093EF0B809174
:104D4000EF0B9091F00B08950F931F93CF93DF9388
:104D5000FC012081318121153105D1F1EC01822F37
:104D60000E94EE3A21E0892B09F420E02B876A8526
:104D7000261729F01E821F82188619860BC08E8185
:104D80009F81A885B9850196A11DB11D8E839F8342
:104D9000A887B9870E811F81288539858A819B81E3
:104DA000AC81BD81081719072A073B078CF081E009
:104DB000682788810E94163B0990D881C02DA7DF03
:104DC00040E050E0BE01DF91CF911F910F914CCE9A
:104DD000DF91CF911F910F9108952F923F924F92A3
:104DE0005F926F927F928F929F92AF92BF92CF927B
:104DF000DF92EF92FF920F931F93CF93DF93CDB784
:104E0000DEB766970FB6F894DEBF0FBECDBF8C013C
:104E10000E94691EF801E550FE4F81E04091220892
:104E2000509123086091240870912508452B462B4A
:104E3000472B09F480E080830E94691EF801E4504A
:104E4000FE4F81E040912608509127086091280884
:104E500070912908452B462B472B09F480E080836D
:104E60000E94691EF801E350FE4F81E040912A083C
:104E700050912B0860912C0870912D08452B462BE2
:104E8000472B09F480E080830E94691E809172089C
:104E900090917308A0917408B0917508F801E250E0
:104EA000FE4F80839183A283B3830E94691E809109
:104EB000760890917708A0917808B0917908F80168
:104EC000EE5FFD4F80839183A283B3830E94691EAE
:104ED00080917A0890917B08A0917C08B0917D0820
:104EE000F801EA5FFD4F80839183A283B3830E9420
:104EF000691E80914A0890914B08A0914C08B0918E
:104F00004D08F801EA5EFD4F80839183A283B3834D
:104F10000E94691E80914E0890914F08A091500800
:104F2000B0915108F801E65EFD4F80839183A28322
:104F3000B3830E94691E8091520890915308A091FA
:104F40005408B0915508F801E25EFD4F80839183CB
:104F5000A283B3830E94691E80915A0890915B08D6
:104F6000A0915C08B0915D08F801EE5DFD4F808373
:104F70009183A283B3830E94691E80915E08909101
:104F80005F08A0916008B0916108F801EA5DFD4FEB
:104F900080839183A283B3830E94691E80916208FB
:104FA00090916308A0916408B0916508F801E65DEE
:104FB000FD4F80839183A283B3830E94691E8091F9
:104FC000FA079091FB07A091FC07B091FD07F8014B
:104FD000E25DFD4F80839183A283B3830E94691EAB
:104FE0008091FE079091FF07A0910008B091010801
:104FF000F801EE5CFD4F80839183A283B3830E940E
:10500000691E8091020890910308A0910408B09154
:105010000508F801EA5CFD4F80839183A283B38386
:105020000E94691EF801E65CFD4F81E02091D207E5
:105030003091D3072130310509F080E080830E9450
:10504000691EF801E55CFD4F81E02091D6073091A3
:10505000D7072130310509F080E080830E94691E66
:10506000F801E45CFD4F81E02091DA073091DB0725
:105070002130310509F080E080830E94691EF8012B
:10508000E85AFD4F81E04091AA075091AB0760912B
:10509000AC077091AD07452B462B472B09F480E0F8
:1050A00080830E94691EF801E75AFD4F81E040911C
:1050B000AE075091AF076091B0077091B107452BD3
:1050C000462B472B09F480E080830E94691EF8017B
:1050D000E65AFD4F81E04091B2075091B3076091CD
:1050E000B4077091B507452B462B472B09F480E098
:1050F00080830E94691EF801E55AFD4F81E04091CE
:105100008208509183086091840870918508452B2E
:10511000462B472B09F480E080830E94691EF8012A
:10512000E45AFD4F81E040918608509187086091D4
:10513000880870918908452B462B472B09F480E09D
:1051400080830E94691EF801E35AFD4F81E040917F
:105150008A0850918B0860918C0870918D08452BBE
:10516000462B472B09F480E080830E94691EF801DA
:10517000E25AFD4F81E02091BA073091BB07213000
:10518000310509F080E080830E94691EF801E15A30
:10519000FD4F81E02091BE073091BF0721303105DE
:1051A00009F080E080830E94691EF801E05AFD4FFB
:1051B00081E02091C2073091C3072130310509F009
:1051C00080E080830E94691E80918207909183070E
:1051D000A0918407B0918507F801EF59FD4F8083B6
:1051E0009183A283B3830E94691E80918607909168
:1051F0008707A0918807B0918907F801EB59FD4F07
:1052000080839183A283B3830E94691E80918A0761
:1052100090918B07A0918C07B0918D07F801E75909
:10522000FD4F80839183A283B3830E94691EF8019E
:10523000E45BFD4F81E040919207509193076091AC
:10524000940770919507452B462B472B09F480E076
:1052500080830E94691EF801E35BFD4F81E040916D
:105260009607509197076091980770919907452B81
:10527000462B472B09F480E080830E94691EF801C9
:10528000E25BFD4F81E040919A0750919B0760914E
:105290009C0770919D07452B462B472B09F480E016
:1052A00080830E94691E80918A0990918B09A09148
:1052B0008C09B0918D09F801E35CFD4F80839183E7
:1052C000A283B3830E94691E80918E0990918F09F9
:1052D000A0919009B0919109F801EF5BFD4F808397
:1052E0009183A283B3830E94691E80919209909159
:1052F0009309A0919409B0919509F801EB5BFD4FDA
:1053000080839183A283B3830E94691EF801E15BCD
:10531000FD4F81E02091EA073091EB072130310504
:1053200009F080E08083F801E05BFD4F1082319648
:1053300010820E94691EF801EE5AFD4F81E0209113
:10534000E6073091E7072130310509F080E08083DE
:10535000F801ED5AFD4F1082319610820E94691EAD
:10536000F801EB5AFD4F81E020910A0830910B08BB
:105370002130310509F080E080830E94691EF80128
:10538000EA5AFD4F81E020910E0830910F0821303C
:10539000310509F080E080830E94691EF801E95A16
:1053A000FD4F81E020911208309113082130310522
:1053B00009F080E080830E94691EF801E75BFD4FE1
:1053C00081E020919A0930919B092130310509F043
:1053D00080E080830E94691EF801E65BFD4F81E05A
:1053E00020919E0930919F092130310509F080E01C
:1053F00080830E94691EF801E55BFD4F81E02091EA
:10540000A2093091A3092130310509F080E08083A1
:105410000E94691E380123E9621A2DEF720A8091F9
:10542000320890913308A0913408B0913508F30107
:1054300080839183A283B3830E94691E5801FFE891
:10544000AF1AFDEFBF0A8091360890913708A091FE
:105450003808B0913908F50180839183A283B38322
:105460000E94691E80913A0890913B08A0913C08E7
:10547000B0913D0898012B583D4FF90180839183ED
:10548000A283B383F3014081518162817381141639
:1054900015061606170644F041E050E060E070E0A3
:1054A0004083518362837383F5014081518162811E
:1054B0007381141615061606170644F041E050E0F5
:1054C00060E070E04083518362837383181619068D
:1054D0001A061B064CF081E090E0A0E0B0E0F90174
:1054E00080839183A283B383D901CD90DD90ED9029
:1054F000FC90F50180809180A280B380D3014D9013
:105500005D906D907C900E94A606FC0140825182C5
:105510006282738284829582A682B782C086D18697
:10552000E286F386F801E75BFD4FB081B9833C97D3
:1055300020813181428153812F87388B498B5A8B4F
:10554000789630813E83399630803F9740814A87F4
:1055500033962080399650815C87339780818B8782
:105560007E973081FF972081EA59FF4F408151811A
:1055700062817381F397C080D180E280F3803C9791
:1055800080809180A280B3803C974080518062806F
:105590007380789780819181A281B381F80180A77F
:1055A00091A7A2A7B3A7D80144A655A666A677A639
:1055B00080AA91AAA2AAB3AAC4AAD5AAE6AAF7AABF
:1055C00040AF51AF62AF73AF24AF35AF2B8525A38A
:1055D0003C8536A337A240E450E060E070E0E05C38
:1055E000FF4F4083518362837383DE962C92DE9754
:1055F000EA85DF96EC93F801EC5BFF4F2E81208368
:1056000031968F859889A989BA8980839183A283ED
:10561000B383349699819083D80155968D919C914E
:1056200056978633910559F482E591E1F19691837D
:10563000808332961182108280E591E11EC08C3306
:10564000910569F48AE491E1F801E658FF4F9183EE
:10565000808332961182108288E491E10EC08E9789
:1056600091F482E491E1F801E658FF4F9183808341
:105670003296118210828CE391E136969183808379
:10568000329611821082F801838D948D4A9789F4A5
:105690008EE491E1E258FF4F91838083329611822C
:1056A00010828CE491E13696918380833296118248
:1056B0001082F801E65BFD4F2081298339978081B4
:1056C0009181A281B3818E839F83A887B9877596C4
:1056D00090819A87399690813F97A081AB873396C6
:1056E000B081BC8739962080339730807E97808147
:1056F000FF9720812F87E759FF4F20813181428119
:1057000053812B8B3C8B4D8B5E8BF397408151816A
:10571000628173813C97C080D180E280F3803C97A6
:1057200080809180A280B380E059F140380132E05E
:10573000630E731ED3014D905D906D907C90408EF2
:10574000518E628E738E848E958EA68EB78EC0A279
:10575000D1A2E2A2F3A244A355A366A377A32B8907
:105760003C894D895E8920A731A742A753A73F8571
:1057700034A785A7358A268A978B80E490E0A0E03D
:10578000B0E080AB91ABA2ABB3AB4C8546A75B85D9
:1057900057A78A8584AB2E813F814885598525ABE3
:1057A00036AB47AB50AF398131AF858196818633B7
:1057B000910579F482E591E1D801AC50BF4F119683
:1057C0009C938E93129611961C921E9280E591E105
:1057D00022C08C33910579F48AE491E1D801AC5070
:1057E000BF4F11969C938E93129611961C921E9207
:1057F00088E491E110C08E97A9F482E491E1D80188
:10580000AC50BF4F11969C938E93129611961C929A
:105810001E928CE391E1169611969C938E931296AC
:105820001D921C92838594854A9791F48EE491E1B0
:10583000F801E850FF4F91838083329611821082E5
:105840008CE491E1369691838083329611821082A6
:10585000F801E55BFD4F4081498336978081918156
:10586000A281B3818E839F83A887B9877296908126
:105870009A873996A081AA833F97B081BB873396D8
:1058800020812C8739962080339730807E97308115
:10589000FF972081E459FF4F80819181A281B381DC
:1058A000F39740815181628173813C97C080D180A0
:1058B000E280F3803C9780809180A280B380EA519F
:1058C000F140FE87ED87EE5FFE4F408051806280A1
:1058D0007380ED85FE85408E518E628E738E848E30
:1058E000958EA68EB78EC0A2D1A2E2A2F3A244A347
:1058F00055A366A377A380A791A7A2A7B3A724A7C0
:1059000035A7358A268A2A81278B80E490E0A0E09B
:10591000B0E080AB91ABA2ABB3AB2C8526A73B85A7
:1059200037A74A8544AB8E819F81A885B98585AB11
:1059300096ABA7ABB0AF298121AF85819681863325
:10594000910569F482E591E1F801E259FE4F9183F6
:10595000808332961182108280E591E11EC08C33E3
:10596000910569F48AE491E1F801E259FE4F9183CF
:10597000808332961182108288E491E10EC08E9766
:1059800091F482E491E1F801E259FE4F9183808322
:105990003296118210828CE391E136969183808356
:1059A000329611821082AD85BE851B968D919C9199
:1059B0001C974A9791F48EE491E1F801EE58FE4F5E
:1059C000918380833296118210828CE491E1369625
:1059D00091838083329611821082F801E45BFD4F3F
:1059E0002081C8014096222319F00E94661602C049
:1059F0000E945216F801E35BFD4F2081C8018657D3
:105A00009F4F222319F00E94661602C00E94521670
:105A1000F801E25BFD4F80818823E1F08D859E8552
:105A200066960FB6F894DEBF0FBECDBFDF91CF9163
:105A30001F910F91FF90EF90DF90CF90BF90AF90AC
:105A40009F908F907F906F905F904F903F902F909E
:105A50000C9466168D859E8566960FB6F894DEBF0B
:105A60000FBECDBFDF91CF911F910F91FF90EF90AF
:105A7000DF90CF90BF90AF909F908F907F906F906E
:105A80005F904F903F902F900C9452160F931F935E
:105A9000CF93DF93FC01E759FF4F20812223C9F008
:105AA0007A9700811181228133813896408151811A
:105AB00062817381041715072607370728F1EC0167
:105AC0000E94E115CE01DF91CF911F910F910C94AF
:105AD0007A17FC01E15AFF4F20812223A9F0709729
:105AE000008111812281338134964081518162810C
:105AF0007381041715072607370730F0DF91CF9120
:105B00001F910F910C941117DF91CF911F910F915D
:105B10000895FC01E15AFF4F2081222361F0709724
:105B200080819181A281B3810196A11DB11D8083E5
:105B30009183A283B38308952F923F924F925F92F5
:105B40006F927F928F929F92AF92BF92CF92DF928D
:105B5000EF92FF920F931F93CF93DF93CDB7DEB7F2
:105B600062970FB6F894DEBF0FBECDBF8C017C01EB
:105B700026E4E20EF11CD7018C919801205A3F4F88
:105B8000F801EF59FF4F6F01A801425C5F4F4A01D6
:105B900014971D01882341F0F80184A5D9018C9345
:105BA00081E0F60180832FC0DA014D915D916D9106
:105BB0007C91F10180819181A281B381BB24B39456
:105BC000481759076A077B070CF0B12CF901B0821E
:105BD00077FF07C070956095509541955F4F6F4F67
:105BE0007F4FB7FF07C0B095A095909581959F4FC7
:105BF000AF4FBF4F21E0481759076A077B070CF4E6
:105C000020E0D6012C93F40140815181628173819F
:105C1000411551056105710559F4F801848D958D83
:105C2000A68DB78DE55AFF4F80839183A283B383FE
:105C3000F10180819181A281B381F80142AC53AC22
:105C400064AC75AC9801215A3F4F5901481659066A
:105C50006A067B0634F4481759076A077B077CF00D
:105C60000AC084159505A605B7052CF48417950779
:105C7000A607B70724F0D7018C918823E9F0F50136
:105C800080818823C9F0D7018C91811105C0F7016B
:105C90008081811111C007C060E0C8010E94F31625
:105CA0008111F5CF19C0D6016C9181E06827C80138
:105CB0000E94F316882381F0D5011C9260E0C80190
:105CC0000E94F316882309F4C5C1F801FE961082DC
:105CD000118212821382BEC1D80194962D913D91FA
:105CE0004D915C91979729833A834B835C835896B7
:105CF0002D913D914D915C915B972D833E834F8318
:105D000058875C962D913D914D915C915F972987C5
:105D10003A874B875C87F10180819181A281B381B1
:105D2000F801FE96C080D180E280F380F80142AD98
:105D300053AD64AD75ADED59FF4F108231961082B1
:105D40003801F5E66F0E711CF301108298012A5993
:105D50003F4FF9011082329610824C015D01841A86
:105D6000950AA60AB70AB7FE08C0B094A09490940A
:105D70008094811C911CA11CB11C481759076A070B
:105D80007B072CF4C41AD50AE60AF70A04C0C81A1D
:105D9000D90AEA0AFB0AD501C401B595A7959795DA
:105DA00087958D879E87AF87B88BD801A859BF4F3D
:105DB0001D01F7FC05C08C149D04AE04BF0464F4FF
:105DC000F80100A0F1A1E02DFA8BE98B81E0D90167
:105DD0008C93F1018083B9C02D853E854F8558890C
:105DE0002C153D054E055F0508F450C089819A8148
:105DF000AB81BC818C159D05AE05BF0544F4AD811A
:105E0000BE811196BA8BA98B81E0F3019BC0C701BB
:105E1000B6010E944A4C2B013C0169817A818B8139
:105E20009C810E944A4C9B01AC01C301B2010E94BB
:105E3000384E2B013C016D817E818F8198852985AB
:105E40003A854B855C85621B730B840B950B0E9416
:105E50004A4C9B01AC01C301B2010E94A94C2B0129
:105E60003C0169857A858B859C850E944A4C9B0103
:105E7000AC01C301B2010E94D44D0E94A04E7A8BA6
:105E8000698B81E0F801ED59FF4F5CC0D501C40179
:105E900029813A814B815C81821B930BA40BB50B4A
:105EA000C816D906EA06FB065CF44D815E814E5F9A
:105EB0005F4F5A8B498B81E0F801EB59FF4F42C08D
:105EC000C501B4016C197D098E099F090E944A4CD5
:105ED0002B013C0169817A818B819C810E944A4C13
:105EE0009B01AC01C301B2010E94384E2B013C0161
:105EF0006D817E818F81988529853A854B855C856A
:105F0000621B730B840B950B0E944A4C9B01AC01E6
:105F1000C301B2010E94A94C2B013C0169857A851D
:105F20008B859C850E944A4C9B01AC01C301B20148
:105F30000E94D44D0E94A04E7A8B698B81E0F801BB
:105F4000EC59FF4F8083D1018C93F8018481882321
:105F5000B1F00E94C33BD80112964D905C9013970C
:105F6000052C000C66087708DC01CB018419950923
:105F7000A609B709893E9340A105B10568F4F80167
:105F8000E55AFF4F29893A89C901A0E0B0E0808332
:105F90009183A283B38392CE0E94C33BD801139610
:105FA0007C936E93129784E294E00E9459398FE1BA
:105FB00096E00E94593960E070E0CB010E94F93907
:105FC00085E296E00E945939C701B6010E94F9396D
:105FD0008BE296E00E945939C501B4010E94F9395B
:105FE00081E396E00E9459394AE06D857E858F8570
:105FF00098890E94B43988E396E00E9459396981F2
:106000007A818B819C810E94F9398EE396E00E940F
:10601000593969857A858B859C850E94F93984E494
:1060200096E00E9459396D817E818F8198850E940A
:10603000F9398AE496E00E94593981EE95E00E9490
:10604000593989899A890E94E93A8CE993E00E943A
:10605000593995CF62960FB6F894DEBF0FBECDBF0B
:10606000DF91CF911F910F91FF90EF90DF90CF9034
:10607000BF90AF909F908F907F906F905F904F9068
:106080003F902F9008950F931F93FC01EA5BFF4F01
:106090002081211110C03897008111812281338124
:1060A0003496408151816281738104171507260758
:1060B00037074CF404C0FC0124A5222321F01F91D2
:1060C0000F910C9438161F910F910C941E16FC0121
:1060D000138212821482168215821086178212860B
:1060E00011861486138616861586108A1786128ADC
:1060F000118A148A138ADC01A15ABF4F1C9212AE76
:1061000013AE14AE15AE91971D921D921D921C9266
:10611000139714961D921D921D921C92139714961C
:106120001C925A961C9211961C9212961C921196D1
:106130001C9211961C9211961C9211961C9211960B
:106140001C9211961C9211968CE292E111969C93EE
:106150008E93129611961C921E92129687E292E1ED
:1061600011969C938E93129611961C921E921296E3
:1061700082E292E111969C938E93129611961C9254
:106180001E9212968DE192E18D939C93E858FF4FF9
:106190001182108208952F923F924F925F926F92D8
:1061A0007F928F929F92AF92BF92CF92DF92EF92A7
:1061B000FF920F931F93CF93DF9300D000D0CDB702
:1061C000DEB79E838D834B015A013A8329831801E0
:1061D000FC82EB82FA01408051806280738020E073
:1061E00030E0A901C301B2010E94D14E181674F427
:1061F000F6012081318142815381C301B2010E94A5
:10620000D34DF5016083718382839383ED81FE8199
:10621000E05AFF4F8081F401068D178DC088D18828
:10622000E288F388F1014080518062807380D80158
:10623000A7019601882341F00E949C4D64157505C5
:106240008605970544F023C00E949C4D46165706CC
:1062500068067906E4F4F50140805180628073801D
:1062600020E030E04AEF56E4C301B2010E94444C02
:1062700087FF0DC020E030E040E85FE3C301B201DA
:106280000E94D44DF5016083718382839383D8018A
:10629000A70196010E949C4DF10160837183828366
:1062A00093838D819E81CE969E838D83FC01808118
:1062B0009181A281B381E981FA8180839183A28354
:1062C000B383EB81FC8180819181892B49F0C401EA
:1062D0000E946E15ED81FE816083718382839383BA
:1062E00026960FB6F894DEBF0FBECDBFDF91CF91DB
:1062F0001F910F91FF90EF90DF90CF90BF90AF90E4
:106300009F908F907F906F905F904F903F902F90D5
:1063100008950E94A6060C940E070E94A6060C94EF
:10632000C205CF93DF93EC01FC01E652FD4F1082D2
:10633000EE58F1098081811104C0CE0140960E947F
:106340005216FE01E35BFD4F8081811105C0CE0135
:1063500086579F4F0E945216FE01E25BFD4F8081DF
:10636000811105C0CE018C5F9E4F0E94521664E6DB
:1063700070E080E090E0DF91CF910C948B3B2F9206
:106380003F924F925F926F927F928F929F92AF92C5
:10639000BF92CF92DF92EF92FF920F931F93CF9312
:1063A000DF93EC010E94691EFE01ED55FD4F8091C7
:1063B000120990911309918380830E94691EFE0146
:1063C000EB55FD4F809116099091170991838083B9
:1063D0000E94691EFE01E955FD4F80911A099091B6
:1063E0001B09918380830E94691E8E0107551D4FF2
:1063F00060913A0970913B0980913C0990913D0967
:106400000E944A4CF80160837183828393830E94C7
:10641000691E1E01F3E52F1AFDEF3F0A60913E0948
:1064200070913F0980914009909141090E944A4C26
:10643000F10160837183828393830E94691E20E04F
:1064400030E048EC52E4F8016081718182819381EF
:106450000E94384E2B013C0120E030E048EC52E431
:10646000F10160817181828193810E94384E4B01DC
:106470005C016091420970914309809144099091B7
:1064800045090E944A4C20E030E048EC52E40E946A
:10649000384E6B017C012AE037ED43E25CE3C30137
:1064A000B2010E94D14E18168CF420E030E046EC88
:1064B00052E4C301B2010E94444C87FD0FC0412C3D
:1064C000512C46EC642E42E4742E08C05AE0452E4E
:1064D00057ED552E53E2652E5CE3752EF801408290
:1064E0005182628273822AE037ED43E25CE3C501A8
:1064F000B4010E94D14E18168CF420E030E046EC36
:1065000052E4C501B4010E94444C87FD0FC0812CA8
:10651000912C26ECA22E22E4B22E08C03AE0832E63
:1065200037ED932E33E2A32E3CE3B32EF1018082AC
:106530009182A282B3822AE037ED43E25CE3C70195
:10654000B6010E94D14E18168CF420E030E046ECE3
:1065500052E4C701B6010E94444C87FD0FC0C12C14
:10656000D12C86ECE82E82E4F82E08C09AE0C92EE1
:1065700097EDD92E93E2E92E9CE3F92EFE01EF541C
:10658000FD4FC082D182E282F3820E94691E809117
:10659000FA089091FB08FE01E854FD4F9183808337
:1065A0000E94691E8091FE089091FF08FE01E6544A
:1065B000FD4F918380830E94691E80910209909112
:1065C0000309FE01E454FD4F918380830E94691EFC
:1065D0008091220990912309A0912409B091250965
:1065E000FE01E254FD4F80839183A283B3830E9416
:1065F000691E8091260990912709A0912809B091E0
:106600002909FE01EE53FD4F80839183A283B3835A
:106610000E94691E80912A0990912B09A0912C0952
:10662000B0912D09FE01EA53FD4F80839183A2832F
:10663000B3830E94691E80914A0990914B09FE0123
:10664000E653FD4F918380830E94691E80914E091D
:1066500090914F09FE01E453FD4F918380830E9486
:10666000691E8091520990915309FE01E253FD4F3A
:10667000918380830E94691E8091620990916309D1
:10668000FE01E053FD4F918380830E94691E80913B
:10669000660990916709FE01EE52FD4F9183808358
:1066A0000E94691E80916A0990916B09FE01EC526B
:1066B000FD4F918380830E94691E8091EA0890912A
:1066C000EB08A091EC08B091ED08FE01EB54FD4FF2
:1066D0000197A105B10519F481E0808301C0108202
:1066E0000E94691E8091EE089091EF08A091F00839
:1066F000B091F108FE01EA54FD4F0197A105B105E3
:1067000019F481E0808301C010820E94691E80918B
:10671000F2089091F308A091F408B091F508C954DB
:10672000DD4F0197A105B10519F481E0888301C00F
:106730001882DF91CF911F910F91FF90EF90DF9022
:10674000CF90BF90AF909F908F907F906F905F9011
:106750004F903F902F9008952F923F924F925F92CB
:106760006F927F928F929F92AF92BF92CF92DF9261
:10677000EF92FF920F931F93CF93DF93CDB7DEB7C6
:10678000A1970FB6F894DEBF0FBECDBF99A388A323
:106790001B010E94ED2688A199A1F1DD88A199A194
:1067A000B8DD88A199A1B9DD21E022163104D9F123
:1067B00032E02316310409F468C02114310409F0D1
:1067C00097C0A8A0B9A040E1A40EB11C88A199A1CE
:1067D00082589E4F9E838D83E8A1F9A1E85AFD4F10
:1067E00090819B87E8A1F9A1E758FD4FF887EF83D7
:1067F00028A139A12D553D4F3D872C8748A159A18E
:106800004B545D4F598B488B88A199A18B509E4F5B
:106810009A878987EDE8F0E0FF87EE8725E130E091
:106820003C832B8368C0A8A0B9A03AE8A30EB11C92
:1068300048A159A140565E4F5E834D83E8A1F9A15E
:10684000E75AFD4F50815B8788A199A183589D4FDE
:1068500098878F83E8A1F9A1EB55FD4FFD87EC8761
:1068600028A139A12A543D4F398B288B48A159A121
:1068700049505E4F5A8749878EE890E09F878E8700
:10688000E6E1F0E0FC83EB8336C0A8A0B9A0FCEF02
:10689000AF1AFEEFBF0A28A139A12E533E4F3E8307
:1068A0002D83E8A1F9A1E65AFD4F30813B8748A12D
:1068B00059A14F575D4F58874F8388A199A189559A
:1068C0009D4F9D878C87E8A1F9A1E954FD4FF98B75
:1068D000E88B28A139A127503E4F3A8729874FE8F6
:1068E00050E05F874E8787E190E09C838B8303C0F5
:1068F00080E596E00CC0C5010E940D16811105C00F
:10690000C5010E94FC15882369F08DEC96E0D1D476
:106910000E94A60681E090E090934507809344078B
:1069200090E0C9C384E294E0C4D48FE796E0C1D478
:10693000F501808159D583E097E0BBD48CE993E0E1
:10694000B8D481E090E0E985FA859183808341E0C5
:1069500050E0B50188A199A10E946223C5010E945F
:106960006616F50184A58501005A1F4F882339F06A
:10697000C5010E94381681E0F801808305C0C50179
:106980000E941E16F80110828D819E810E946E1554
:10699000F501FE966083718382839383EF81F8858E
:1069A0001082118212821382E8A1F9A1E758FD4FEB
:1069B0001082118212821382E8A1F9A1E358FD4FDF
:1069C0001082118212821382E8A1F9A1EF57FD4FC4
:1069D000108211821282138286E090E0E985FA85A6
:1069E0009183808346E050E0B50188A199A10E947F
:1069F000622341E050E0B50188A199A10E9445239E
:106A0000412C512C3201439488A199A1820D931DF0
:106A10009C012B543D4F3B8B2A8B4101880C991CC8
:106A2000880C991CC40187559D4F48A159A1480F56
:106A3000591F5F8B4E8BC1018B599E4F880F991F39
:106A4000E8A1F9A1E80FF91FF98FE88FC401895671
:106A50009D4F28A139A1280F391F3B8F2A8FA401F0
:106A600045575D4F5D8F4C8F88A199A1880D991D69
:106A7000FC01EE5DFD4FFF8FEE8FEA89FB8980817F
:106A80008823B9F0A40147585D4F28A139A1420FCE
:106A9000531FCE88DF88E88CF98C0A8D1B8D2C8DD6
:106AA0003D8D88A199A1280F391F6D817E81C50177
:106AB00072DB87EF9BE00E9431101816190624F054
:106AC0001A82198210E01CC087EF9BE00E940F1011
:106AD0008F7D85349105A1F78DEE94E0EAD30E9475
:106AE000A60621E0FC01248782E693E0E2D30E941F
:106AF000A6060E94B00521E030E03A83298311E028
:106B0000C5010E940D168111C3C2C5010E94FC156A
:106B10008111BEC21111BCC2EC85FD8560817181FD
:106B2000072E000C880B990B0E944A4C9B01AC016C
:106B3000EF81F88560817181828193810E94444C4C
:106B400087FFA6C2C5010E94111708A119A1080D4F
:106B5000191D0E5D1D4FF801208131814281538145
:106B600060E573EC80E090E00E94764DC901C8D5E5
:106B7000F8012081318142815381A3E0B0E00E947D
:106B8000924D9B01AC01C301B2010E94764D672B6F
:106B9000682B692B39F48EE593E08BD30E94A6060F
:106BA0000E94B005C5010E94E115EE8DFF8D208188
:106BB00031814281538160E573EC80E090E00E9476
:106BC000764DC9019DD5FFEF4F1A5F0A6F0A7F0A04
:106BD00029813A81232B09F450CF41E050E05A83B8
:106BE000498342E050E0B50188A199A10E94452364
:106BF00084E294E05ED38FE796E05BD3F501808179
:106C0000F3D386E896E055D38CE993E052D32981FB
:106C10003A81232BD1F489E996E04BD381EE95E0BC
:106C200048D387E196E045D38B819C81D2D481EE15
:106C300095E03FD389E196E03CD33B85832F90E0FC
:106C4000C8D40E94A6060E94B00588A199A161DB64
:106C500088A199A162DB84E294E02BD38FE796E0D0
:106C600028D3F5018081C0D38DE996E022D38CE949
:106C700093E01FD3EF81F885108211821282138274
:106C8000F50184A58501005A1F4F882331F0C50105
:106C90000E941E16F801108206C0C5010E94381617
:106CA00081E0F80180838D819E810E946E15F5013F
:106CB000FE966083718382839383E8A1F9A1E758EC
:106CC000FD4F1082118212821382E8A1F9A1E358CC
:106CD000FD4F1082118212821382E8A1F9A1EF57B1
:106CE000FD4F10821182128213828D819E810E943B
:106CF0006E156A8B7B8B8C8B9D8B8D819E810E9408
:106D00006E15412C512C32014394812C912C88A179
:106D100099A1820D931D9C012B543D4F3F8B2E8BCF
:106D2000A101440F551F440F551F5C834B83CA01BB
:106D300087559D4FE8A1F9A1E80FF91FF98FE88F5A
:106D4000C1018B599E4F880F991F28A139A1280F87
:106D5000391F3B8F2A8FCA0189569D4F48A159A1DF
:106D6000480F591F5D8F4C8F8B819C81E8A1F9A141
:106D70008E0F9F1F9C012E5D3D4F3F8F2E8F4981AF
:106D80005A81452B09F0C5C0EE89FF89808188238F
:106D9000D1F02B813C8125573D4F48A159A1240FAB
:106DA000351F4B815C8147585D4F88A199A1480FE1
:106DB000591FC88CD98CEA8CFB8C0C8D1D8D6D8174
:106DC0007E81C501E8D987EF9BE00E94311018163B
:106DD000190614F010E01CC087EF9BE00E940F1012
:106DE0008F7D85349105B1F78DEE94E062D20E94DB
:106DF000A60621E0FC01248782E693E05AD20E9495
:106E0000A6060E94B00521E030E03A83298311E014
:106E10003AE08316910434F4EF81F88510821182F0
:106E200012821382FB85C501F1113EC10E94FC153F
:106E300081113DC111113BC1EC85FD8560817181DE
:106E4000072E000C880B990B0E944A4C9B01AC0149
:106E5000EF81F88560817181828193810E94444C29
:106E600087FF25C1C5010E941117FFEF8F1A9F0AE6
:106E70000B811C8128A139A1020F131F0E5D1D4F2C
:106E8000F801208131814281538160E573EC80E01B
:106E900090E00E94764DC90133D4F8012081318100
:106EA00042815381A3E0B0E00E94924D9B01AC016E
:106EB000C301B2010E94764D672B682B692B91F4B8
:106EC0008EE593E0F6D10E94A6060E94B00584E20A
:106ED00094E0EFD181EB96E0ECD1C4017AD38CE958
:106EE00093E0E7D1C5010E94E115EE8DFF8D208171
:106EF00031814281538160E573EC80E090E00E9433
:106F0000764DC901FDD3FFEF4F1A5F0A6F0A7F0A62
:106F100036CF21E030E03A83298384E294E0C9D17E
:106F20008FE796E0C6D1F50180815ED28FEB96E0C7
:106F3000C0D18CE993E0BDD18D819E810E946E15F8
:106F400028893989232BA1F0DC01CB012A893B89CF
:106F50004C895D89821B930BA40BB50BB7FF07C04F
:106F6000B095A095909581959F4FAF4FBF4F4C0125
:106F700049815A81452BF9F489E996E09AD181EE4D
:106F800095E097D187E196E094D18E859F8521D3B6
:106F900081EE95E08ED189E196E08BD1B401092C88
:106FA000000C880B990B0E944A4C42E049D20E9487
:106FB000A6060E94B00585E090E0E985FA859183F8
:106FC000808345E050E0B50188A199A10E94622329
:106FD000C5010E94521688A199A19BD988A199A1A7
:106FE0009CD9F1E02F163104A9F022E022163104D9
:106FF00001F1232861F50E94A606C401990CAA0B91
:10700000BB0B80934A0790934B07A0934C07B09318
:107010004D071DC00E94A606C401990CAA0BBB0B0C
:1070200080934E0790934F07A0935007B09351075A
:107030000EC00E94A606C401990CAA0BBB0B80933C
:10704000520790935307A0935407B09355070E949B
:10705000A6060E940306E985FA851182108240E0A7
:1070600050E0B50188A199A10E94622340E050E060
:10707000B50188A199A10E9445230E94A6062981F5
:107080003A81309345072093440789819A8113C040
:1070900082E297E00ED1C5010E94FC15882309F415
:1070A000A0CDF1E0FB879DCD0E940D16C1CE82E2FE
:1070B00097E0FFD032CFA1960FB6F894DEBF0FBE97
:1070C000CDBFDF91CF911F910F91FF90EF90DF9097
:1070D000CF90BF90AF909F908F907F906F905F9078
:1070E0004F903F902F9008950F931F93CF93DF936E
:1070F000FC01E851FE4F208131812115310509F451
:1071000046C0EC018C0104511E4FF8018081918131
:10711000CC51DE4F82179307D0F428813981211595
:10712000310561F0F901E80FF91F80818A3041F0E3
:107130008D3029F48CE993E0BCD002C080E054D1BA
:10714000F8018081918101969183808320C060E065
:1071500070E0CE010E9486122881398181110DC014
:107160002115310519F0C9010E946B471982188257
:107170001D821C821B821A8207C01D821C826EE93E
:1071800073E0C9010E94E64FF80111821082DF917D
:10719000CF911F910F91089590E0FC013197E2315A
:1071A000F10508F04EC08827EC59FE4F8F4F0C9424
:1071B000E54E809180008F7703C0809180008F7DA5
:1071C00080938000089580918000877FF9CF84B5F7
:1071D0008F7702C084B58F7D84BD08958091B00003
:1071E0008F7703C08091B0008F7D8093B0000895A9
:1071F000809190008F7707C0809190008F7D03C0B1
:1072000080919000877F8093900008958091A000E6
:107210008F7707C08091A0008F7D03C08091A00070
:10722000877F8093A0000895809120018F7707C009
:10723000809120018F7D03C080912001877F809302
:10724000200108953FB7F89480913E0D90913F0D35
:10725000A091400DB091410D26B5A89B05C02F3FD0
:1072600019F00196A11DB11D3FBFBA2FA92F982F6C
:107270008827820F911DA11DB11DBC01CD0142E0E7
:10728000660F771F881F991F4A95D1F708950097B9
:1072900069F0FC0101900020E9F73197AF01481B2C
:1072A000590BBC0187EF9BE00C94D20F80E090E07B
:1072B0000895EDCFEF92FF920F931F93CF93DF933B
:1072C000CDB7DEB764970FB6F894DEBF0FBECDBF63
:1072D0007C01CB01BA018E010F5F1F4F22E044E019
:1072E0000E94B446FC0101900020E9F73197AF01FC
:1072F000481B590BBC01C7010E94AD1264960FB622
:10730000F894DEBF0FBECDBFDF91CF911F910F91DB
:10731000FF90EF900895CF93DF93EC0119821882CC
:107320001B821A821D821C8260E070E00E9486121D
:107330002881398181110FC02115310519F0C9014A
:107340000E946B47198218821D821C821B821A823E
:10735000DF91CF9108951D821C826EE973E0C9010F
:10736000DF91CF910C94E64F8F929F92AF92BF9294
:107370000F931F93CF93DF93CDB7DEB7A1970FB6CF
:10738000F894DEBF0FBECDBF19A2423008F44AE028
:107390008E010F5D1F4F842E912CA12CB12CA501C5
:1073A00094010E94A24DE62FB901CA0101501109B2
:1073B000EA3014F4E05D01C0E95CD801EC93232BC2
:1073C000242B252B61F7C80162DFA1960FB6F89434
:1073D000DEBF0FBECDBFDF91CF911F910F91BF9048
:1073E000AF909F908F900895682F87EF9BE00C944B
:1073F0006810CF92DF92EF92FF92CF93DF9397FFC7
:1074000017C06B017C018DE2EFDFEC016627772767
:10741000CB016C197D098E099F094AE0A5DF8C0F0D
:107420009D1FDF91CF91FF90EF90DF90CF90089557
:107430004AE0DF91CF91FF90EF90DF90CF9094CF13
:107440008F929F92AF92BF92CF92DF92EF92FF9274
:107450000F931F93CF93DF936B017C01142F9B013C
:10746000AC010E94D54E882319F086E397E027C02F
:1074700046015701E894B7F82FEF3FEF4FE75FE77A
:10748000C501B4010E94D54E81110DC02FEF3FEF11
:107490004FE75FE7C501B4010E94444C18161CF485
:1074A0008AE397E00CC02FEF3FEF4FE75FE4C7019F
:1074B000B6010E94D14E18167CF48EE397E0DF915E
:1074C000CF911F910F91FF90EF90DF90CF90BF90E1
:1074D000AF909F908F90DBCE2FEF3FEF4FE75FECA9
:1074E000C701B6010E94444C87FDE7CF20E030E0A1
:1074F000A901C701B6010E94444C87FF08C08DE274
:1075000073DFEC01F7FAF094F7F8F09402C0C0E0F2
:10751000D0E000E060E070E080E09FE3101741F011
:1075200020E030E040E251E40E94384E0F5FF6CF99
:10753000A70196010E94D44D6B017C010E94A54ECB
:107540004B015C014AE010DFC80FD91F112399F1EC
:10755000C501B4010E94484C9B01AC01C701B601B2
:107560000E94D34D6B017C018EE23EDFC80FD91F14
:1075700020E030E040E251E4C701B6010E94A94C8E
:107580004B015C010E94A54E6B01E12CF12C4AE0FD
:10759000C701B601E9DEC80FD91FC701B6010E94B5
:1075A000484C9B01AC01C501B4010E94D34D6B0155
:1075B0007C011150E9F6CE01DF91CF911F910F911F
:1075C000FF90EF90DF90CF90BF90AF909F908F9003
:1075D0000895BC01990F880B990B0BCFCF93DF93C4
:1075E000282F30E0F901E550FB4F8491F901EB546D
:1075F000FB4FD491F901E159FB4FC491CC2389F0A1
:107600008111CADDEC2FF0E0EE0FFF1FEB5AFB4FAC
:10761000A591B491EC91ED2381E090E021F480E01C
:1076200002C080E090E0DF91CF9108951F93CF9347
:10763000DF93282F30E0F901E550FB4F8491F901E9
:10764000EB54FB4FD491F901E159FB4FC491CC238A
:10765000B9F0162F8111A0DDEC2FF0E0EE0FFF1F27
:10766000E55CFB4FA591B4919FB7F894111104C04C
:107670008C91D095D82302C0EC91DE2BDC939FBF78
:10768000DF91CF911F910895CF93DF9390E0FC019C
:10769000EB54FB4F2491FC01E159FB4F849188236B
:1076A00061F190E0880F991FFC01EF5DFB4FC591E0
:1076B000D491FC01E55CFB4FA591B491611109C027
:1076C0009FB7F8948881209582238883EC912E239C
:1076D0000BC0623061F49FB7F8948881322F3095E7
:1076E00083238883EC912E2B2C939FBF06C08FB7EA
:1076F000F894E8812E2B28838FBFDF91CF910895D6
:107700008230910538F0880F991F880F991F0597CF
:107710000197F1F708958F929F92AF92BF92CF9207
:10772000DF92EF92FF926B017C018CDD4B015C01DB
:10773000C114D104E104F104E9F084DDDC01CB01E2
:1077400088199909AA09BB09883E9340A105B1058A
:1077500078F321E0C21AD108E108F10888EE880E1A
:1077600083E0981EA11CB11CC114D104E104F104F2
:1077700021F7DECFFF90EF90DF90CF90BF90AF90DA
:107780009F908F9008952FB7F89460913A0D709163
:107790003B0D80913C0D90913D0D2FBF08951F92A0
:1077A0000F920FB60F9211242F933F938F939F93B5
:1077B000AF93BF9380913A0D90913B0DA0913C0DFA
:1077C000B0913D0D3091390D23E0230F2D3720F47A
:1077D0000196A11DB11D05C026E8230F0296A11D2B
:1077E000B11D2093390D80933A0D90933B0DA093DA
:1077F0003C0DB0933D0D80913E0D90913F0DA091B9
:10780000400DB091410D0196A11DB11D80933E0D1B
:1078100090933F0DA093400DB093410DBF91AF9158
:107820009F918F913F912F910F900FBE0F901F90BE
:107830001895789484B5826084BD84B5816084BDD8
:1078400085B5826085BD85B5816085BD80916E00FE
:10785000816080936E00109281008091810082602F
:10786000809381008091810081608093810080916C
:1078700080008160809380008091B100846080935B
:10788000B1008091B00081608093B0008091910040
:10789000826080939100809191008160809391003B
:1078A000809190008160809390008091A10082601F
:1078B0008093A1008091A10081608093A1008091BC
:1078C000A00081608093A00080912101826080935C
:1078D000210180912101816080932101809120010B
:1078E00081608093200180917A00846080937A0087
:1078F00080917A00826080937A0080917A00816022
:1079000080937A0080917A00806880937A00109248
:10791000C10061E086E3B8DE61E087E3B5DE61E0E7
:1079200086E2B2DE61E08AE1AFDE61E08CE1ACDEEE
:1079300061E088E1A9DE62E083E0A6DE62E082E049
:10794000A3DE62E080E1A0DE62E081E19DDE62E034
:107950008FE19ADE62E081E297DE61E08CE394DE03
:1079600061E08DE391DE61E088E38EDE62E08EE02F
:107970008BDE62E08FE088DE62E087E185DE62E038
:1079800089E182DE62E083E27FDE62E085E27CDE26
:1079900061E08EE279DE61E080E376DE61E08EE335
:1079A00073DE62E082E170DE62E083E16DDE62E060
:1079B0008BE16ADE62E08DE167DE62E087E264DE31
:1079C00062E089E261DE61E08AE05EDE61E088E03B
:1079D0005BDE61E089E058DE61E08DE055DE62E06B
:1079E0008FE352DE62E08BE34FDE62E088E24CDE42
:1079F00062E080E449DE62E08AE246DE62E08CE238
:107A000043DE62E081E440DE62E082E43DDE62E08B
:107A100084E33ADE62E085E337DE62E080E034DE74
:107A200062E081E031DE62E089E32EDE62E08AE33B
:107A30002BDE62E081E328DE62E082E325DE62E0A5
:107A400083E322DE62E08BE21FDE62E08DE21CDE79
:107A500062E08FE219DE62E080E216DE61E084E03F
:107A600013DE61E085E010DE61E086E00DDE61E0BE
:107A70008BE00ADE61E086E2D9DD61E088E1D6DDF7
:107A800061E088E3D3DD61E08EE3D0DDE091070CB7
:107A9000F091080C82E08083E091030CF091040CDB
:107AA0001082E091050CF091060CD0E1D083109289
:107AB0000F0CE0910B0CF0910C0C86E08083E091B0
:107AC000090CF0910A0C808180618083E091090C9F
:107AD000F0910A0C808188608083E091090CF0911C
:107AE0000A0C808180688083E091090CF0910A0C77
:107AF00080818F7D808364E670E080E090E00BDE23
:107B00000E94AC240E94DD1F0E9408250E94D824F8
:107B10003ADE81E392E19093430780934207C1E00C
:107B2000C0936F00D093810010928000C093DA0A56
:107B300080E092E0909387008093860081E18093BB
:107B40008100109281001092850010928400809133
:107B5000DA0A80618093810016DE6093D80B7093FF
:107B6000D90B8093DA0B9093DB0B0DDE0CDE609368
:107B7000DC0B7093DD0B8093DE0B9093DF0B0E9488
:107B8000691E80915E0790915F07A0916007B09198
:107B900061070197A105B10579F40E94691E8091E2
:107BA000A6079091A707A091A807B091A9070197F0
:107BB000A105B10509F4EBC70E94691E80915E071B
:107BC00090915F07A0916007B09161070197A105AF
:107BD000B10579F40E94691E8091A2079091A307D4
:107BE000A091A407B091A5070197A105B10509F4DB
:107BF000EDC70E94691E80915E0790915F07A0917A
:107C00006007B09161070197A105B10579F40E9461
:107C1000691E80919E0790919F07A091A007B09147
:107C2000A1070197A105B10509F4F0C780E893E029
:107C300040DBEFE72E2EE2E03E2EF9E86F2EF2E079
:107C40007F2EA1DD0091DC0B1091DD0B2091DE0B6E
:107C50003091DF0B601771078207930748F4609338
:107C6000DC0B7093DD0B8093DE0B9093DF0B2EC04B
:107C7000AB01BC01401B510B620B730B483E5340E0
:107C80006105710518F1D901C80188519C4FAF4FAA
:107C9000BF4F8093DC0B9093DD0BA093DE0BB09372
:107CA000DF0B0E940825EC010E94A426CE010C9651
:107CB0000E94A426CE0148960E94A426CE01849656
:107CC0000E94A426CE01C0960E94A42687EF9BE0C6
:107CD0000E943110892B09F4B7C555DD6093D80B8C
:107CE0007093D90B8093DA0B9093DB0B87EF9BE0BB
:107CF0000E940F108093D70B982F9F7D953479F0B9
:107D00002091D50B3091D60BF901EF58F44F8083B9
:107D10002F5F3F4F3093D60B2093D50B06C00E94A8
:107D2000A60621E0DC011C962C938091D50B909146
:107D3000D60B8336910564F02AE02093D70BFC0123
:107D4000EF58F44F208301969093D60B8093D50B78
:107D50008091D70B2091D50B3091D60B8A3021F032
:107D6000243631050CF470C5C9010197ACE0BBE0C5
:107D7000E1E7FBE0AF0141575B40481759071CF4AE
:107D800041914D93F7CFFC01E45FF44F1082223014
:107D900031050CF455C581E193E08BDA81EE95E075
:107DA00088DA8FE993E085DA8CE09BE082DA8FE96C
:107DB00093E07FDA8CE993E07CDA8AE390E0F3D712
:107DC000EC011A821B821C821D821E821F82188671
:107DD00019861A861B861C861D861E861F86188A93
:107DE000198A1A8A1B8A1C8A1D8A1E8A1F8A188E63
:107DF000198E1A8E1B8E1C8E1D8E1E8E1F8E18A223
:107E000019A21AA21BA21CA21DA21EA21FA218A682
:107E100019A61AA61BA61CA61DA61EA61FA618AA52
:107E200019AA1AAA1BAA1CAA1DAA1EAA1FAA18AE22
:107E300019AE68E072E08CE09BE00E94F7478C018D
:107E4000FC0180818654823008F027C161EA73E02A
:107E5000C8010E94DD4F892B09F4D3C064EA73E0A6
:107E6000C8010E94DD4F892B09F4CBC068EA73E09A
:107E7000C8010E94DD4F892B09F4C6C06BEA73E08C
:107E8000C8010E94DD4F892B09F4BEC06FEA73E080
:107E9000C8010E94DD4F892B09F4B9C063EB73E080
:107EA000C8010E94DD4F892B09F4B4C067EB73E071
:107EB000C8010E94DD4F892B09F4ACC06AEB73E066
:107EC000C8010E94DD4F892B09F4A7C06EEB73E057
:107ED000C8010E94DD4F892B09F4A2C062EC73E057
:107EE000C8010E94DD4F892B09F49DC066EC73E048
:107EF000C8010E94DD4F892B09F498C06AEC73E039
:107F0000C8010E94DD4F892B09F493C06EEC73E029
:107F1000C8010E94DD4F892B09F48EC062ED73E029
:107F2000C8010E94DD4F892B09F489C066ED73E01A
:107F3000C8010E94DD4F892B09F484C06AED73E00B
:107F4000C8010E94DD4F892B09F47FC06EED73E0FC
:107F5000C8010E94DD4F892B09F47AC062EE73E0FC
:107F6000C8010E94DD4F892B09F475C066EE73E0ED
:107F7000C8010E94DD4F892B09F470C06AEE73E0DE
:107F8000C8010E94DD4F892B09F46BC06EEE73E0CF
:107F9000C8010E94DD4F892B09F466C062EF73E0CF
:107FA000C8010E94DD4F892B09F461C066EF73E0C0
:107FB000C8010E94DD4F892B09F45CC06AEF73E0B1
:107FC000C8010E94DD4F892B09F457C06EEF73E0A2
:107FD000C8010E94DD4F892B09F452C062E074E0B1
:107FE000C8010E94DD4F892B09F44DC066E074E0A2
:107FF000C8010E94DD4F892B09F048C088EB90E052
:1080000047C080E090E044C081E090E041C08CE156
:1080100090E03EC08DE690E03BC08FE690E038C037
:1080200080E790E035C081E790E032C082E790E0E1
:108030002FC083E790E02CC084E790E029C088E758
:1080400090E026C089E790E023C08AE790E020C056
:1080500083E890E01DC084E890E01AC08DE890E0CD
:1080600017C08EE890E014C08FE890E011C080E95E
:1080700090E00EC081EA90E00BC085EB90E008C074
:1080800086EB90E005C087EB90E002C08FEF9FEF9A
:108090009093010280930002BBC08FEF9FEF9093FB
:1080A000010280930002B8C0D8018C91883539F460
:1080B000C801019699D76A837B838C839D83F801DD
:1080C0008081893539F4C80101968ED76E837F830C
:1080D00088879987D8018C918A3539F4C80101962F
:1080E00083D76A877B878C879D87F801808181345D
:1080F00049F4C801019678D70E94A04E6E877F8709
:10810000888B998BD8018C91823449F4C8010196EF
:108110006BD70E94A04E6A8B7B8B8C8B9D8BF8015A
:108120008081833449F4C80101965ED70E94A04E35
:108130006E8B7F8B888F998FD8018C91833539F422
:10814000C801019651D76A8F7B8F8C8F9D8FF80164
:108150008081803549F4C801019646D70E94A04E1F
:108160006E8F7F8F88A399A3D8018C91863549F4AF
:10817000C801019639D70E94A04E6AA37BA38CA3A5
:108180009DA3F8018081873549F4C80101962CD759
:108190000E94A04E6EA37FA388A799A7D8018C91B7
:1081A000853449F4C80101961FD70E94A04E6AA7E2
:1081B0007BA78CA79DA7F8018081843549F4C8016D
:1081C000019612D70E94A04E6EA77FA788AB99ABED
:1081D000D8018C918D3449F4C801019605D70E94CD
:1081E000A04E6AAB7BAB8CAB9DABF8018081813537
:1081F00049F4C8010196F8D60E94A04E6EAB7FAB41
:1082000088AF99AF6AE074E080E090E0F0D68C012E
:108210000115110509F048CF0E94A606DC011C9645
:108220001C910E94691E80906A0790906B07A09035
:108230006C07B0906D07CEA8DFA8E8ACF9AC0E943F
:10824000A606C0924607D0924707E0924807F092F0
:108250004907809100029091010255245394823085
:10826000910538F09C012F5631092630310508F070
:10827000512C112371F08D36910559F09C0128572E
:1082800031092330310528F0855B9109039708F007
:10829000CDC20E94691E80915E0790915F07A091F8
:1082A0006007B09161070197A105B10529F055203C
:1082B00019F08DEF92E0BCC2209719F489EF92E09B
:1082C000B7C2E0900002F0900102BFEFEB16FB0690
:1082D000A9F3E114F104B9F48091030B9091040B1C
:1082E000892B61F482E090E05ED523EE32E0FC0160
:1082F000318320839093040B8093030B0091030B35
:108300001091040B6EC0FCE1EF16F104B9F48091FA
:10831000010B9091020B892B61F482E090E043D530
:108320002FEC32E0DC012D933C939093020B809371
:10833000010B0091010B1091020B53C0BDE6EB162F
:10834000F104B9F48091FF0A9091000B892B61F43C
:1083500082E090E028D525EC32E0FC0131832083D7
:108360009093000B8093FF0A0091FF0A1091000B7D
:1083700053C0FFE6EF16F104B9F48091FD0A909125
:10838000FE0A892B61F482E090E00DD52BEB32E000
:10839000DC012D933C939093FE0A8093FD0A00919B
:1083A000FD0A1091FE0A53C0B0E7EB16F104B9F4D0
:1083B0008091FB0A9091FC0A892B61F482E090E0A5
:1083C000F2D421EB32E0FC01318320839093FC0A4C
:1083D0008093FB0A0091FB0A1091FC0A6CC000E03C
:1083E00010E0F1E7EF16F104B9F48091F90A9091E9
:1083F000FA0A892B61F482E090E0D5D427EA32E0D2
:10840000DC012D933C939093FA0A8093F90A009132
:10841000F90A1091FA0A68C0B2E7EB16F104B9F450
:108420008091F70A9091F80A892B61F482E090E03C
:10843000BAD42DE932E0FC01318320839093F80A0D
:108440008093F70A0091F70A1091F80A68C0F3E7E1
:10845000EF16F104B9F48091F50A9091F60A892B90
:1084600061F482E090E09FD423E932E0DC012D93B7
:108470003C939093F60A8093F50A0091F50A1091C7
:10848000F60A68C0B4E7EB16F104A9F48091F30A88
:108490009091F40A892B51F482E090E084D4FC019D
:1084A000718260829093F40A8093F30A0091F30A38
:1084B0001091F40A6AC0F8E7EF16F104A9F480916C
:1084C000F10A9091F20A892B51F482E090E06BD48A
:1084D000DC012D923C929093F20A8093F10A009174
:1084E000F10A1091F20A6CC0B9E7EB16F104B9F485
:1084F0008091EF0A9091F00A892B61F482E090E07C
:1085000052D425E732E0FC01318320839093F00AB6
:108510008093EF0A0091EF0A1091F00A6CC03AE7DD
:10852000E316F104B9F48091ED0A9091EE0A892BDB
:1085300061F482E090E037D4EBE6F2E0DC01ED9309
:10854000FC939093EE0A8093ED0A0091ED0A10914E
:10855000EE0A6CC0FDE8EF16F104B9F48091EB0A65
:108560009091EC0A892B61F482E090E01CD4E1E662
:10857000F2E0DC01ED93FC939093EC0A8093EB0A1C
:108580000091EB0A1091EC0A6CC0FEE8EF16F104C2
:10859000B9F48091E90A9091EA0A892B61F482E0AA
:1085A00090E001D4E7E5F2E0DC01ED93FC939093D9
:1085B000EA0A8093E90A0091E90A1091EA0A6CC07C
:1085C000FFE8EF16F104B9F48091E70A9091E80A08
:1085D000892B61F482E090E0E6D3EDE4F2E0DC0187
:1085E000ED93FC939093E80A8093E70A0091E70AE1
:1085F0001091E80A6CC0F0E9EF16F104B9F480912B
:10860000E50A9091E60A892B61F482E090E0CBD3F1
:10861000E3E4F2E0DC01ED93FC939093E60A8093AF
:10862000E50A0091E50A1091E60A6CC0F1EAEF163E
:10863000F104B9F48091E30A9091E40A892B61F482
:1086400082E090E0B0D3E9E3F2E0DC01ED93FC934B
:108650009093E40A8093E30A0091E30A1091E40AFC
:108660006BC0F5EBEF16F104B9F48091E10A90913B
:10867000E20A892B61F482E090E095D3EFE2F2E028
:10868000DC01ED93FC939093E20A8093E10A009160
:10869000E10A1091E20A50C0F6EBEF16F104B9F4CA
:1086A0008091DF0A9091E00A892B61F482E090E0EA
:1086B0007AD3E5E2F2E0DC01ED93FC939093E00ADB
:1086C0008093DF0A0091DF0A1091E00A35C0F7EBD2
:1086D000EF16F104B9F48091DD0A9091DE0A892B3E
:1086E00061F482E090E05FD3EBE1F2E0DC01ED9336
:1086F000FC939093DE0A8093DD0A0091DD0A1091CD
:10870000DE0A1AC0F8EBEF16F104B1F48091DB0A2F
:108710009091DC0A892B61F482E090E044D3E1E19E
:10872000F2E0DC01ED93FC939093DC0A8093DB0A8A
:108730000091DB0A1091DC0A0115110589F489EF1B
:1087400092E00E9459390E94A6060E94B0058EE070
:1087500094E00E9447398CE993E00E9447396EC04B
:1087600085EF92E00E9459390E94A6060E94B0054A
:108770000E94A6061092450710924407E12CF12CA6
:108780002FEFE21AF20A31E0E316F10441F081EF33
:1087900092E00E9459390E94A6060E94B005D801B5
:1087A000ED91FC910480F581E02DBE01C801199581
:1087B0000E94A606C0904407D09045070E94A606D6
:1087C000FC01848581110AC0E814F9043CF4C11449
:1087D000D10421F0F2E0CF16D10491F687EF9BE0AF
:1087E0000E943110181619062CF487EF9BE00E94A6
:1087F0000F10F4CFCD2809F42CC2552009F426C25D
:108800000E94691E8091660790916707A091680792
:10881000B09169070197A105B10509F017C20E943F
:10882000A60621E0DC011C962C9310C281E093E0A7
:108830000E9459390E94A6060E94B005CE014BD372
:108840001092D60B1092D50B80910B0B8111A6C004
:108850000E94A606FC018485882309F49FC00E941B
:10886000AC24EC01FC01E652FD4F108240960E94C0
:108870005216CE0186579F4F0E945216CE018C5F32
:108880009E4F0E9452160E9487267C018C01C1E0F7
:10889000D0E0D80111968C918823D9F084E294E03D
:1088A0000E94593988E294E00E945939CE010E9411
:1088B000E93A8CE993E00E94593960E08C2F0E94DC
:1088C000163B40E050E0BE01C7010E943425F8018C
:1088D0001182D801D9968C918823F9F084E294E032
:1088E0000E9459398FE394E00E945939CE010E94C9
:1088F000E93A8CE993E00E94593961E08C2F0E949B
:10890000443B60E08C2F0E94163B41E050E0BE01EA
:10891000C7010E943425F80111AE21960F5F1F4F49
:10892000C533D10509F0B5CF0E94C52480912D0D26
:1089300090E09C01220F331F820F931FFC01E4562D
:10894000F34F80818F7B80838091300D90E09C017C
:10895000220F331F820F931FFC01E456F34F8081D7
:108960008F7B80838091330D90E09C01220F331F19
:10897000820F931FFC01E456F34F80818F7B80832D
:108980008091360D90E09C01220F331F820F931FC0
:10899000FC01E456F34F80818F7B80830E94A60602
:1089A000DC011C968C9180930B0B0E94691E209118
:1089B000090B30910A0BFC0182819381281739073A
:1089C00099F00E94691EDC0112968D919C9113977B
:1089D00090930A0B8093090B0E94AC240E94DD1F28
:1089E0000E9408250E94D8240E94C33B0091D80B06
:1089F0001091D90B2091DA0B3091DB0B60177107C6
:108A00008207930708F4B6C0DC01CB01801B910BF1
:108A1000A20BB30B89389341A105B10508F4B4C08A
:108A20000E94A606DC011C968C91882319F08DE02B
:108A300093E002C089E093E00E9459390E94A606A3
:108A40000E94B0050E94AC24EC01FC01EB54FD4FE8
:108A50008081882341F0CE0182589E4F0E946E157E
:108A60006B017C0107C0FE01E25BFF4FC080D1803B
:108A7000E280F3800E94A606C0924A07D0924B077C
:108A8000E0924C07F0924D07FE01EA54FD4F8081C1
:108A9000882341F0CE0180569E4F0E946E156B01D7
:108AA0007C0107C0FE01E853FF4FC080D180E28007
:108AB000F3800E94A606C0924E07D0924F07E09224
:108AC0005007F0925107FE01E954FD4F8081882341
:108AD00041F0CE018E539E4F0E946E156B017C01BA
:108AE00006C0CE5BDE4FC880D980EA80FB800E9442
:108AF000A606C0925207D0925307E0925407F09214
:108B000055070E94A6060E9403060E94AC240E94FC
:108B1000F3230E94A6060E940E070E94A6060E944A
:108B2000C2050E94691E80915E0790915F07A09127
:108B30006007B09161070197A105B10541F085E09B
:108B400093E00E9459390E94A6060E94B0058091C8
:108B5000050B9091060BA091070BB091080B0196A5
:108B6000A11DB11D8093050B9093060BA093070BDD
:108B7000B093080B0E94C33B6093D80B7093D90B42
:108B80008093DA0B9093DB0B0E94D5105AC885E5D1
:108B900094E00E9459390E94AC24CF931F921F92F7
:108BA0001F921F92812C912CA12CB12CC12CD12C65
:108BB000760197018601B701A6010E9480070F90F8
:108BC0000F900F900F900F900C94DC3D8DE694E089
:108BD0000E9459390E94AC241F9221E02F931F92CA
:108BE0001F921F92812C912CA12CB12CC12CD12C25
:108BF000760197018601B701A6010E9480070F90B8
:108C00000F900F900F900F900C94F93D85E894E031
:108C10000E9459390E94AC241F921F9221E02F9389
:108C20001F921F92812C912CA12CB12CC12CD12CE4
:108C3000760197018601B701A6010E9480070F9077
:108C40000F900F900F900F900C94163E89EE92E0CB
:108C500002C08DEE92E00E9459390E94A6060E9441
:108C6000B0050E94A6061092460710924707109280
:108C7000480710924907E2CD8091940C9091950C91
:108C80002AC11092FA0B1092F90B88EE93E0A0E043
:108C9000B0E08093FB0B9093FC0BA093FD0BB09383
:108CA000FE0B8AE693E09093F80B8093F70B85EC2C
:108CB00090E09093040C8093030C84EC90E09093EC
:108CC000060C8093050C80EC90E09093080C809348
:108CD000070C81EC90E090930A0C8093090C82ECD5
:108CE00090E090930C0C80930B0C86EC90E09093AA
:108CF0000E0C80930D0C1092100C1092110C10920F
:108D0000120C1092130C82E090E04DD02CE733E06F
:108D1000FC013183208390939B0C80939A0C84E90F
:108D20009CE00E948B3980912C0DADE2BDE09FEF5D
:108D300048EB5BE0803378F48C93282F30E0F90126
:108D4000EE0FFF1F2E0F3F1FF901E456F34F528322
:108D500041838F5F01C09C931396FDE0A933BF0749
:108D600049F780932C0D0895EF920F931F93CF93A3
:108D7000DF93E80147FD02C034E001C034E1042E76
:108D8000000C550B57FF03C0519541955109E32E37
:108D9000022F242FAE01A7D1CE01DF91CF911F91D9
:108DA0000F91EF9008950F931F93CF93DF9382302D
:108DB000910510F482E090E0E091460DF091470DAE
:108DC00020E030E0A0E0B0E0309719F1408151811F
:108DD0000281138148175907C8F08417950769F471
:108DE000109731F012960C93129713961C9327C08C
:108DF0000093460D1093470D22C02115310519F03F
:108E00004217530718F49A01BD01EF01DF01F80181
:108E1000DBCF21153105F9F0281B390B2430310542
:108E200080F48A819B816115710521F0FB01938398
:108E3000828304C09093470D8093460DFE013296C5
:108E400044C0FE01E20FF31F819391932250310938
:108E5000398328833AC02091440D3091450D232B4E
:108E600041F420910402309105023093450D209386
:108E7000440D20910202309103022115310541F485
:108E80002DB73EB74091060250910702241B350BC7
:108E9000E091440DF091450DE217F307A0F42E1B6D
:108EA0003F0B2817390778F0AC014E5F5F4F24174E
:108EB000350748F04E0F5F1F5093450D4093440D0A
:108EC0008193919302C0E0E0F0E0CF01DF91CF9178
:108ED0001F910F910895CF93DF93009709F481C0FC
:108EE000FC01329713821282A091460DB091470D7A
:108EF000109781F420813181820F931F2091440DBE
:108F00003091450D2817390751F5F093450DE09341
:108F1000440D67C0ED0120E030E0CE17DF0740F4DC
:108F20004A815B819E0141155105F1F0EA01F5CFBF
:108F3000D383C28340815181840F951FC817D907FD
:108F400059F488819981840F951F029691838083BB
:108F50008A819B81938382832115310529F4F093C3
:108F6000470DE093460D3DC0E901FB83EA8349913B
:108F70005991C40FD51FEC17FD0761F480819181D1
:108F8000840F951F0296E9019983888382819381DA
:108F90009B838A83E0E0F0E012968D919C91139779
:108FA000009719F0FD01DC01F7CF8D919C9111978D
:108FB0009D012E5F3F4F820F931F2091440D3091F2
:108FC000450D2817390769F4309729F41092470D99
:108FD0001092460D02C013821282B093450DA093E9
:108FE000440DDF91CF91089566277727F2C142E4BF
:108FF0005DE000C0FA01A191B081009719F41097CB
:10900000E1F0CD01DC01CD010D90002011F4C00193
:1090100013C0FB012191222319F02015D9F7F3CFBA
:10902000FB012191201519F41E92119606C02223EE
:10903000C1F70D900020A1F7D001FA01A193B083F0
:109040000895BB274A3031F4992322F4BDE290956C
:1090500081959F4F30C0BB272A3051F4992342F4A9
:10906000BDE290958095709561957F4F8F4F9F4F92
:1090700001C0BB27FA01A62F621771058105910572
:10908000330B30FB66F0AA27660F771F881F991FE6
:10909000AA1FA21710F0A21B63953850A9F7A05D74
:1090A000AA3308F0A95DA19336F7B111B1931082EC
:1090B000CA01DAC3BB27FB015527AA27880F991FCE
:1090C000AA1FA41710F0A41B83955051B9F7A05DF7
:1090D000AA3308F0A95DA193009779F7B111B19374
:1090E0001192CB01C1C38F929F92AF92BF92CF9248
:1090F000DF92EF92FF920F931F93CF93DF93CDB741
:10910000DEB729970FB6F894DEBF0FBECDBF6A0158
:10911000122FB02E2BE3201720F0FF24F394F00E33
:1091200002C02CE3F22E0F2D27E0AE014F5F5F4F00
:10913000A3D2BC014981842F8970813031F0E1FCD8
:1091400006C0E0FE06C090E205C09DE203C09BE2BF
:1091500001C090E05E2D507143FF3CC0911102C0F0
:1091600083E001C084E0811718F4212F281B01C07F
:1091700020E051110BC0F601822F30E2882319F054
:1091800031938150FBCFC20ED11C20E0992329F0EE
:10919000D6019C93F60131966F01C6010396E2FE5B
:1091A0000AC03EE4D6013C9341E411964C931197DA
:1091B00012963C9306C03EE6F601308341E64183B9
:1091C0003283FC01322F40E2332309F442C0419341
:1091D0003150FACF42FF44C0911102C083E001C078
:1091E00084E0811718F4212F281B01C020E05111C1
:1091F0000BC0F601822F30E2882319F031938150A1
:10920000FBCFC20ED11C20E0992329F0D6019C93FC
:10921000F60131966F01C6010396E2FE0BC039E4F8
:10922000D6013C933EE411963C93119736E4129696
:109230003C9307C039E6F60130833EE6318336E6DB
:109240003283FC01322F40E2332319F04193315035
:10925000FBCFFC01E20FF11D10828EEF9FEFA6C045
:1092600021E030E0911102C020E030E01616170630
:109270001CF4FB01319602C0E1E0F0E02E0F3F1F2D
:10928000BB2021F0EB2DF0E0319602C0E0E0F0E0F1
:109290002E0F3F1FE12FF0E02E173F071CF4121B8B
:1092A000212F01C020E08E2D887159F4F601822F04
:1092B00030E2882319F031938150FBCFC20ED11CCC
:1092C00020E0992329F0D6019C93F60131966F0195
:1092D00051110BC0F601822F90E3882319F091936E
:1092E0008150FBCFC20ED11C20E00F2D060F9A81BA
:1092F000342F307144FF03C0913309F4015010162C
:1093000024F4093018F008E001C001E0AB0177FF58
:1093100002C040E050E0FB01E41BF50BA1E0B0E02F
:10932000AC0FBD1FEA0FFB1F8EE2A82E4B01801A67
:1093300091080B2D10E01195019511094F3FBFEFDA
:109340005B0721F4D601AC9211966D016417750785
:109350002CF08416950614F4818101C080E34150FD
:1093600051093196D60111967D014017510724F01D
:10937000D6018C936701E2CF6417750739F49633F1
:1093800020F4953319F4311101C081E3F601808393
:10939000F701822F90E2882319F091938150FBCF3F
:1093A000F701E20FF11D108280E090E029960FB6E0
:1093B000F894DEBF0FBECDBFDF91CF911F910F910B
:1093C000FF90EF90DF90CF90BF90AF909F908F90E5
:1093D00008958F929F92AF92BF92CF92DF92EF92B9
:1093E000FF920F931F93CF93DF93EC016B016115F5
:1093F000710519F0FB01918380837E01FFEFEF1A65
:10940000FF0A0881802F90E00FD2892B11F0E7012D
:10941000F4CF0D3239F47E0182E0E80EF11C0981AF
:1094200011E008C00B3229F47E0192E0E90EF11C34
:10943000098110E0E701219743E050E064EF72E01A
:10944000CE01FAD1892BB9F4239645E050E06FEEB6
:1094500072E0CE01F1D1892B09F42596C114D10413
:1094600019F0F601D183C0831111F0C060E070E003
:1094700080E89FE7F4C043E050E06CEE72E0CE017C
:10948000DBD1892B59F4C114D10409F4E4C0F2E012
:10949000EF0EF11CF601F182E082DDC020E030E049
:1094A000A901C0E0D0E0F70160EDA62EA00E89E092
:1094B0008A1528F1912F9260B92E812F887012FFA2
:1094C00004C0811123C0219621C081112197A5E0FC
:1094D000B0E028D3DC01CB01880F991FAA1FBB1F66
:1094E0009C01AD012A0D311D411D511D283989E90D
:1094F0003807480789E1580748F0166006C09EEF14
:10950000A9120AC013FD40C01860B12E8FEFE81AEF
:10951000F80A00811B2DC7CF802F8F7D8534A1F5E0
:1095200080818D3211F4106106C08B3221F03196AA
:1095300061E070E004C08181329662E070E08053A7
:109540008A3018F0E61BF70B1FC060E070E060384F
:109550009CE079075CF4DB01AA0FBB1FAA0FBB1FBD
:109560006A0F7B1F660F771F680F711D3196DF0131
:1095700011978C9180538A3050F314FF03C071957A
:1095800061957109C60FD71F11FF08C0C114D1041E
:1095900029F0CF010197F60191838083CA01B901B7
:1095A00077D1212F2370233019F04B015C0106C0C5
:1095B0004B015C01B7FAB094B7F8B09420E030E00A
:1095C000A901C501B40160D1882309F43CC0D7FFCB
:1095D00006C0D195C195D1090BE013E002C003E2AA
:1095E00013E06801F8E1CF1AD10890E2E92EF12CDE
:1095F000CE15DF056CF0F801259135914591549118
:10960000C501B401A6D14B015C01CE19DF09F0CF31
:1096100004501109F594E7940C151D0549F78A2D9E
:10962000880F8B2D881F8F3F41F020E030E0A9018B
:10963000C501B40129D1811106C082E290E0909366
:10964000490D8093480DC501B40109C060E070E088
:1096500080E89FEF04C060E070E080EC9FE7DF915E
:10966000CF911F910F91FF90EF90DF90CF90BF901F
:10967000AF909F908F900895283008F027E033270F
:10968000DA01990F311D87FD916000966105710522
:1096900039F432602E5F3D9330E32A95E1F7089567
:1096A0009F3F30F080387105610509F03C5F3C5FF9
:1096B0003D93913008F08068911DDF93CF931F9305
:1096C0000F93FF92EF92192F987F9695E92F969519
:1096D0009695E90FFF27EF57FC4F99273327EE2484
:1096E000FF24A701E70105900894079428F4360F9A
:1096F000E71EF81E491F511D660F771F881F991F0F
:109700000694A1F70590079428F4E70EF81E491F68
:10971000561FC11D770F881F991F661F0694A1F75A
:109720000590079428F4F80E491F561FC71FD11D36
:10973000880F991F661F771F0694A1F7059007945D
:1097400020F4490F561FC71FD81F990F661F771F98
:10975000881F0694A9F784911095177041F0D6954B
:10976000C79557954795F794E7941A95C1F7E7E29F
:10977000F3E0689415901591359165919591059058
:109780007FE27395E118F10A430B560BC90BD00920
:10979000C0F7E10CF11E431F561FC91FD01D7EF4F8
:1097A000703311F48A95E6CFE894015030F0080F39
:1097B0000AF40027021708F4202F2395022F7A338A
:1097C00028F079E37D932A95E9F710C07D932A95D7
:1097D00089F6069497956795379517951794E1182C
:1097E000F10A430B560BC90BD00998F023957E91D3
:1097F00073957A3308F070E37C932013B8F77E9169
:1098000070617D9330F0839571E37D9370E32A95C9
:10981000E1F71124EF90FF900F911F91CF91DF910D
:10982000992787FD909508959111F6C0803219F01F
:1098300089508550D0F70895FB01DC01415050401C
:1098400088F08D9181341CF08B350CF4805E65912D
:1098500061341CF06B350CF4605E861B611171F392
:10986000990B0895881BFCCFDC01FC01672F7191D7
:109870007723E1F7329704C07C916D9370836291F6
:10988000AE17BF07C8F3089540D008F481E00895EB
:10989000E89409C097FB3EF490958095709561958A
:1098A0007F4F8F4F9F4F9923A9F0F92F96E9BB2740
:1098B0009395F695879577956795B795F111F8CFBC
:1098C000FAF4BB0F11F460FF1BC06F5F7F4F8F4F27
:1098D0009F4F16C0882311F096E911C0772321F01D
:1098E0009EE8872F762F05C0662371F096E8862FB5
:1098F00070E060E02AF09A95660F771F881FDAF70C
:10990000880F9695879597F90895990F0008550F38
:10991000AA0BE0E8FEEF16161706E807F907C0F0F5
:1099200012161306E407F50798F0621B730B840BFD
:10993000950B39F40A2661F0232B242B252B21F4D7
:1099400008950A2609F4A140A6958FEF811D811D77
:1099500008950BD07BC06CD028F071D018F09523FF
:1099600009F05DC062C01124A5C081D0A0F3959F0D
:10997000D1F3950F50E0551F629FF001729FBB27F6
:10998000F00DB11D639FAA27F00DB11DAA1F649FA2
:109990006627B00DA11D661F829F2227B00DA11D55
:1099A000621F739FB00DA11D621F839FA00D611DDB
:1099B000221F749F3327A00D611D231F849F600DFC
:1099C000211D822F762F6A2F11249F5750408AF035
:1099D000E1F088234AF0EE0FFF1FBB1F661F771FC1
:1099E000881F91505040A9F79E3F510570F017C055
:1099F00061C05F3FECF3983EDCF386957795679501
:109A0000B795F795E7959F5FC1F7FE2B880F911DDE
:109A10009695879597F9089599278827089597F936
:109A20009F6780E870E060E008959FEF80EC089504
:109A300000240A941616170618060906089500242D
:109A40000A9412161306140605060895092E0394A7
:109A5000000C11F4882352F0BB0F40F4BF2B11F41B
:109A600060FF04C06F5F7F4F8F4F9F4F089557FD7A
:109A70009058440F551F59F05F3F71F04795880F7C
:109A800097FB991F61F09F3F79F087950895121613
:109A900013061406551FF2CF4695F1DF08C01616BF
:109AA00017061806991FF1CF869571056105089470
:109AB0000895E894BB2766277727CB0197F9089587
:109AC000F999FECF92BD81BDF89A992780B5089586
:109AD000262FF999FECF1FBA92BD81BD20BD0FB6CA
:109AE000F894FA9AF99A0FBE01960895052E97FBFD
:109AF00016F400940FD057FD05D024D007FC02D0F7
:109B000046F408C050954095309521953F4F4F4FF2
:109B10005F4F089590958095709561957F4F8F4F19
:109B20009F4F089531D0A59F900DB49F900DA49F95
:109B3000800D911D11240895B7FFF4CFF3DF821B30
:109B4000930B0895A1E21A2EAA1BBB1BFD010DC0A9
:109B5000AA1FBB1FEE1FFF1FA217B307E407F507DD
:109B600020F0A21BB30BE40BF50B661F771F881FB9
:109B7000991F1A9469F760957095809590959B014F
:109B8000AC01BD01CF010895A29FB001B39FC001F8
:109B9000A39F700D811D1124911DB29F700D811D19
:109BA0001124911D08955058BB27AA270ED04ECFDF
:109BB0003FDF30F044DF20F031F49F3F11F41EF41A
:109BC00034CF0EF4E095E7FB2ACFE92F50DF80F386
:109BD000BA17620773078407950718F071F49EF5AA
:109BE00068CF0EF4E0950B2EBA2FA02D0B01B90112
:109BF00090010C01CA01A0011124FF27591B99F003
:109C0000593F50F4503E68F11A16F040A22F232F0E
:109C1000342F4427585FF3CF469537952795A7955E
:109C2000F0405395C9F77EF41F16BA0B620B730B05
:109C3000840BBAF09150A1F0FF0FBB1F661F771F76
:109C4000881FC2F70EC0BA0F621F731F841F48F42B
:109C5000879577956795B795F7959E3F08F0B3CFB1
:109C60009395880F08F09927EE0F9795879508959B
:109C70000CD0ECCEE4DE40F0DBDE30F021F45F3FD0
:109C800019F0CDCE511116CFD0CEF1DE98F3992335
:109C9000C9F35523B1F3951B550BBB27AA276217B0
:109CA0007307840738F09F5F5F4F220F331F441FF5
:109CB000AA1FA9F333D00E2E3AF0E0E830D091502D
:109CC0005040E695001CCAF729D0FE2F27D0660F1A
:109CD000771F881FBB1F261737074807AB07B0E859
:109CE00009F0BB0B802DBF01FF2793585F4F2AF06F
:109CF0009E3F510568F093CEDDCE5F3FECF3983E7A
:109D0000DCF3869577956795B795F7959F5FC9F7CB
:109D1000880F911D9695879597F90895E1E0660F54
:109D2000771F881FBB1F621773078407BA0720F0CD
:109D3000621B730B840BBA0BEE1F88F7E095089536
:109D400004D06894B111B6CE089599DE88F09F577B
:109D500090F0B92F9927B751A0F0D1F0660F771F77
:109D6000881F991F1AF0BA95C9F712C0B13081F057
:109D7000A0DEB1E008959DCE672F782F8827B85FC9
:109D800039F0B93FCCF3869577956795B395D9F7B8
:109D90003EF490958095709561957F4F8F4F9F4FC2
:109DA0000895B3DD08F48FEF0895AFDD880B990BAC
:109DB0000895991B79E004C0991F961708F0961B27
:109DC000881F7A95C9F780950895EE0FFF1F881FA9
:109DD0008BBF0790F691E02D19946F927F928F922E
:109DE0009F92AF92BF92CF92DF92EF92FF920F932A
:109DF0001F93CF93DF93009789F4CB01DF91CF912D
:109E00001F910F91FF90EF90DF90CF90BF90AF9098
:109E10009F908F907F906F900C94D346FC01E60F3B
:109E2000F71F9C0122503109E217F30708F4A7C07D
:109E3000EC01D9010D911C91119706171707A8F095
:109E40000530110508F499C0C801049786179707D3
:109E500008F493C002501109061B170B01931193CC
:109E60006D937C93CF0137D888C05B01A01AB10AEB
:109E70004C01800E911EA091460DB091470D612CB2
:109E8000712CE12CF12C109709F446C08D919C9116
:109E90001197A815B905B1F56C0142E0C40ED11CAB
:109EA000CA14DB0478F14C018A189B08640142E073
:109EB000C40ED11C1296BC9012971396AC91B5E0CB
:109EC000CB16D10440F0B282A38391828082D90163
:109ED0006D937C9309C00E5F1F4F800F911FF90196
:109EE00091838083EB2DFA2FE114F10431F0D70137
:109EF0001396FC93EE93129740C0F093470DE093B6
:109F0000460D3BC06816790608F43C017D011296A7
:109F10000D90BC91A02DB7CF8091440D9091450D2F
:109F200088169906E1F466167706C8F48091020255
:109F300090910302009741F48DB79EB740910602BD
:109F400050910702841B950BE817F907C0F4F093B2
:109F5000450DE093440DF901718360830EC0CB0180
:109F60000E94D3467C01009751F0A801BE011CD08D
:109F7000CE010E946B47C70104C0CE0102C080E041
:109F800090E0DF91CF911F910F91FF90EF90DF90C4
:109F9000CF90BF90AF909F908F907F906F900895DB
:109FA00081E090E0F89419C0FB01DC0102C001904F
:109FB0000D9241505040D8F70895FB01DC018D917E
:109FC000019080190110D9F3990B0895FB01DC0170
:109FD00001900D920020E1F7089512E0C2EAD2E06C
:109FE00000E005C0802FFE01F0DE2196011DC33A7E
:0C9FF000D10780E00807B1F7F894FFCF1C
:109FFC00FFFF00004A0D8000200A0D000000000049
:10A00C0000901F731CD31C00000000911F751C5C7A
:10A01C001C000000005B05D702DF06000000005C9E
:10A02C0005D9025507000000005D05DB0216030090
:10A03C000000005E05DD027903000000005F05DF13
:10A04C0002B703000000006005D502F70200000013
:10A05C00006105E1025C03000000006205E302D62A
:10A06C0003000000006305E502C703000000006464
:10A07C0005E702E406000000006505E90223040080
:10A08C000000006605EB025B04000000006705EDB4
:10A09C00029304000000006805EF02CB04000000EE
:10A0AC00006905F102FB04000000006A05F3022BB5
:10A0BC0005000000006B05F5020807000000008E8B
:10A0CC001F6F1CE51E000000008D1F6D1CCA1B00BD
:10A0DC000000008F1F711C771C523033005230323D
:10A0EC00005230370052303100523039005238387B
:10A0FC00005238370052383800523030005238375E
:10A10C00005230380052313300523132005231316A
:10A11C000052373300523732005237310052313748
:10A12C00005231360052313500362E342E322E523A
:10A13C000000010000000100000001000000523886
:10A14C00350052383400523035005230360052301F
:10A15C00340052383700000000006810D20F001095
:10A16C00B41031100F102310000000008C1F6B1C5A
:10A17C005239392041524455494E4F205354415283
:10A18C0054555020434F4D504C4554450D0A002A10
:10A19C00004730004730300047310047303100472E
:10A1AC0032380046303900463900463131004631EC
:10A1BC0032004631330046313400463135004631E9
:10A1CC0036004632300046323100463232004633D9
:10A1DC0031004633320046343100463432004634C6
:10A1EC0033004634340046363100463831004638A8
:10A1FC0032004638330046383400200A0D005239FC
:10A20C00392068616E646C6572203D3D204E554C62
:10A21C004C0D0A00523939002072657365747469EB
:10A22C006E67206469676974616C2070696E0020C8
:10A23C00726573657474696E6720616E616C6F67AB
:10A24C002070696E0052393920484F4D45205A20F4
:10A25C004F4E20535441525455500D0A0052393927
:10A26C0020484F4D452059204F4E205354415254B5
:10A27C0055500D0A0052393920484F4D4520582071
:10A28C004F4E20535441525455500D0A00523939F7
:10A29C00204572726F723A20696E76616C69642027
:10A2AC00706172616D657465722069640D0A0020BD
:10A2BC00510052383100205841002058420020599A
:10A2CC00410020594200205A4100205A4200523885
:10A2DC00320052323000686F6D650D0A0052393908
:10A2EC0020656D657267656E63792073746F700D90
:10A2FC000A00523939206572726F720D0A00523998
:10A30C00392073746F707065640D0A0052393920EE
:10A31C006572726F72200020646561637469766186
:10A32C007465206D6F746F7220582064756520748D
:10A33C006F206D697373656420737465707300208E
:10A34C0064656163746976617465206D6F746F7296
:10A35C0020592064756520746F206D697373656472
:10A36C002073746570730020646561637469766131
:10A37C007465206D6F746F72205A2064756520743B
:10A38C006F206D697373656420737465707300520C
:10A39C0039392074696D656F75742058206178693E
:10A3AC00730D0A005239392074696D656F7574200C
:10A3BC005920617869730D0A005239392074696D1E
:10A3CC00656F7574205A20617869730D0A005238D4
:10A3DC003320005239392057696C6C207A65726FC2
:10A3EC002058005239392057696C6C207A65726F8D
:10A3FC002059005239392057696C6C207A65726F7C
:10A40C00205A005232310050005600523431002094
:10A41C00737461200020637572200020656E6420C7
:10A42C00002068616C662000206C656E2000206D39
:10A43C00696E2000206D617820002073706420000C
:10A44C005239392043616C6962726174696F6E2094
:10A45C006572726F723A20696E76616C6964206104
:10A46C007869732073656C65637465640D0A0020EC
:10A47C00617869732000206174207374617274694F
:10A48C006E6720706F696E74005232330020636106
:10A49C006C6962726174696E67206C656E67746852
:10A4AC0000207374657020636F756E743A20002001
:10A4BC00617420656E6420706F696E740052393956
:10A4CC002043616C6962726174696F6E206572728F
:10A4DC006F723A20656E642073746F7020616374C0
:10A4EC00697665206265666F72652073746172743B
:10A4FC000D0A00206D6F766520746F207374617285
:10A50C007420666F722063616C6962726174696F2A
:10A51C006E00523939206D6F76656D656E742064EE
:10A52C006F6E650D0A006E616E00696E66006F7667
:02A53C006600B7
:00000001FF
